:020000040800F2
:10000000C8100020050100083B3800084D290008F1
:1000100039380008350F0008C160000800000000F2
:10002000000000000000000000000000054700087C
:10003000BD1A000800000000AD3D0008ED490008B1
:100040001F010008AD3B00081F0100081F01000848
:100050001F0100081F0100081F0100081F01000800
:100060001F0100081F0100081F0100081F010008F0
:100070001F0100081F010008791500081F01000872
:100080001F0100081F010008410700081F010008A8
:100090001F0100081F0100081F0100081F010008C0
:1000A0005D4A00083D4B00081F0100081F010008C1
:1000B000414B0008314E00088D5000081F01000818
:1000C0001F0100081F0100081F0100081F01000890
:1000D0001F010008B95B00081F0100081F0100088C
:1000E0001F0100081F0100081F010008DFF810D0E1
:1000F00000F0E8FA00480047D9710008AFF300802B
:10010000C81000200648804706480047FEE7FEE783
:10011000FEE7FEE7FEE7FEE7FEE7FEE7FEE7FEE7B7
:100120000D4A0008ED0000082DE9F0410024061BEF
:10013000254671F1000605DA01240027D0EB0700FF
:1001400067EB0101161E73F1000605DA0027D2EBFA
:100150000702012567EB030300F0D0F986460E463F
:1001600017469C46AC4204D00025D0EB050E65EB4B
:10017000010624B10020D2EB000760EB030C7046AF
:1001800031463A466346BDE8F08140EA01039B07E9
:1001900003D009E008C9121F08C0042AFAD203E0FC
:1001A00011F8013B00F8013B521EF9D2704780EA7A
:1001B000010210B502F00043400022D04A001FD0D7
:1001C000010E01EB1261C0F35600C2F3560240F477
:1001D000000042F40002A0FB022000047F39140456
:1001E00000D0401C50EA124001D44000491EC2B267
:1001F0000C0604EBD010401C4008802A02D003E01B
:10020000002010BD20F00100002900DA0020184372
:1002100010BD2DE9FE4F81EA030404F0004421F0F3
:10022000004100944FF0000B23F0004350EA01041A
:100230005ED052EA03045BD0C3F30A54C1F30A55FB
:100240002C44A4F2F3340194A0FB0254C1F3130133
:1002500041F48011C3F3130343F4801301FB024400
:1002600000FB034E840A970A44EA815447EA835705
:10027000A4FB076802958D0A05FB07854FEA932CBE
:1002800004FB0C542705029D4FEA065847EA16372F
:10029000B5EB08056EEB070C870E920E47EA811747
:1002A00042EA8312A7FB0201B6EB0B0164EB0004E8
:1002B0002B0D43EA0C335E1844EB1C50DA465146D2
:1002C000E7FB0201C5F313044FEA0B3343EA14536F
:1002D0004FEA0432019C43EA0603A4F10C040294A1
:1002E000009CCDE900B400F09FF903B0BDE8F08FA9
:1002F00000200146F9E72DE9F04D81EA030404F0FE
:10030000004B21F0004514464FF0000A23F0004155
:1003100050EA050220D054EA01021DD0C5F30A5765
:100320000246C5F31303C1F31300C1F30A5640F4A8
:10033000801543F48013A7EB0608101BD64608F27D
:10034000FD3873EB050002D308F1010801E09218B3
:100350005B41B8F1000F03DA00200146BDE8F08DE3
:1003600000204FF48011064684460EE0171B73EB05
:10037000050705D3121B63EB050306434CEA010C8A
:1003800049084FEA300092185B4150EA0107EDD16D
:1003900052EA030012D082EA040083EA050108430E
:1003A00005D0101BAB4106D20122002306E000223B
:1003B0004FF0004302E06FF0010253101AEB060009
:1003C0004CEB085110EB0A0041EB0B01BDE8F04D7E
:1003D00000F01BB970B521F0004303430CD0C1F30A
:1003E0000A550024D5EB040564EB0403D617AD1AB7
:1003F000B34102DB0020014670BD201841EB0251E1
:1004000070BDC10F80EAE0700844CA07962300213E
:1004100000F0CDB896230022114600F0C8B80EB502
:10042000C10F80EAE0700844CA07002140F233435C
:100430008DE80E000A460B4600F0F6F803B000BD4A
:100440000EB540F2334102910021CDE900110A4678
:100450000B4600F0E9F803B000BD00F0004220F0C8
:100460000040C10DC0F3160040F400007F2901DAFE
:1004700000207047962903DCC1F19601C84001E0D5
:1004800096398840002AF4D04042704770B5C1F3D5
:100490000A5201F000450024C1F3130140F2FF337A
:1004A00041F480119A4201DA002070BD40F23343DA
:1004B0009A42A2F2334203DC524200F05FF800E0BD
:1004C00090402C43F1D0404270BDC1F30A5210B5A8
:1004D000C1F3130140F2FF3341F480119A4201DA73
:1004E000002010BD40F233439A42A2F2334203DCB3
:1004F000524200F043F810BD904010BD2DE9F05F6E
:100500000546002092469B46884606468146402482
:100510001BE0284641464746224600F02FF8534646
:100520005A46C01A914110D311461846224600F08F
:1005300016F82D1A67EB01084F46224601200021CC
:1005400000F00DF817EB00094E41201EA4F1010444
:10055000DFDC484631462A464346BDE8F09F202A64
:1005600004DB203A00FA02F1002070479140C2F10A
:10057000200320FA03F3194390407047202A04DB3C
:10058000203A21FA02F00021704721FA02F3D0400C
:10059000C2F1200291400843194670470029A8BFC4
:1005A0007047401C490008BF20F00100704710B49C
:1005B000B0FA80FC00FA0CF050EA010404BF10BC51
:1005C000704749B1CCF1200421FA04F411FA0CF17E
:1005D00018BF012121430843A3EB0C01CB1D4FEAB7
:1005E00000614FEA102042BF002010BC704700EBB2
:1005F000C35010440029A4BF10BC7047401C4900E0
:1006000008BF20F0010010BC704710B5141E73F134
:10061000000408DA401C41F1000192185B411A43C2
:1006200001D120F0010010BD2DE9F04D92469B460E
:1006300011B1B1FA81F202E0B0FA80F220329046B4
:10064000FFF78DFF04460F4640EA0A0041EA0B011E
:1006500053465A46084313D0114653EA010019D0B5
:10066000C8F140025046FFF789FF05460E46504646
:1006700059464246FFF773FF084305D0012004E0C6
:1006800020463946BDE8F08D0020054346EAE07675
:100690002C4337430A986305E40AA0EB08000022C4
:1006A000FD0A44EA47540A3002D500200146E9E732
:1006B000010510196941DDE9084500196941BDE8E6
:1006C000F04DA2E7064C074D06E0E06840F001035C
:1006D00094E8070098471034AC42F6D3FFF70AFDC0
:1006E000449100086491000870B58C1810F8015B03
:1006F00015F0070301D110F8013B2A1106D110F8BB
:10070000012B03E010F8016B01F8016B5B1EF9D1BE
:100710002B0705D40023521E0DD401F8013BFAE744
:1007200010F8013BCB1A921C03E013F8015B01F8AF
:10073000015B521EF9D5A142D8D3002070BD000044
:1007400070B54E4C4FF490652946204600F019FADA
:10075000002864D02946204600F0A6F848490888B9
:10076000401C08800121204600F0EAFA454942F287
:100770001072B1F85000904202D2401CA1F8500013
:1007800006F00AFF404DB5F91410B5F9120005F056
:10079000CDFD3E4CA5F84A002080A1682046884740
:1007A000A088A5F84C0003F0B1F806F0F7FF384E2A
:1007B000384C3078082833D045F6AC30606042F6CB
:1007C000EF60A06042F2C400E0603348008A2080FD
:1007D000208E6080A16B2F488847208E69882F4C1F
:1007E00008444FF6FF7101EA8000E885207A4FF057
:1007F000000540071DD501F0F1FA294949F6A2404C
:100800000880284840F21A62C188491C89B2C18018
:10081000914204D3A16821F00401A160C58070BD9C
:1008200041F2130060604FF48060A06040F61B50FE
:10083000CAE730780A281BD2DFE800F01A0616054E
:100840000A050D1A1114EAE7BDE8704005F012BF61
:1008500007F04AFE08E0BDE8704002F0A1BD06F0D6
:1008600093FA01E007F0F2F8BDE8704007F0EEB847
:1008700000F0F8FB84F8B65070BD00000024014081
:10088000F0060020340100205C0000200C0700204E
:10089000E7060020C8000020E401002090020020AC
:1008A000442C0140100900206FEA112101607047BB
:1008B0000029816802D041F0010101E021F001012D
:1008C000816070470029816802D041F4807101E0A5
:1008D00021F48071816070472DE9F041824E92B021
:1008E000304600F00BF90BA800F039FA01214FF463
:1008F000C06003F011FB00248DF831404FF46020FC
:10090000CDE90D044FF4A0204FF009080B9001270A
:100910008DF83C808DF830700BA9304600F080F9DE
:10092000724D8DF831408DF830708DF83C700BA908
:10093000284600F075F901231A460F21304600F0D1
:10094000C0F9022201231146304600F0BAF9012312
:1009500003220021304600F0B4F901230422194695
:10096000304600F0AEF9012305220B21304600F09D
:10097000A8F9012306220421304600F0A2F9012340
:1009800007220821304600F09CF9012308220321A8
:10099000304600F096F9012309220A21304600F082
:1009A00090F90121304600F084F90121284600F039
:1009B00080F901231A460521304600F055F901233C
:1009C0001A460621284600F04FF90021304600F073
:1009D000CBF84FF4E041284600F0C6F8012130463C
:1009E00000F0B8F80121284600F0B4F801213046A3
:1009F00000F0A6F80121284600F0A2F801213046B7
:100A000000F09EF90121284600F09AF940F61451B1
:100A1000374804F012FE12208DF8400002208DF8B5
:100A200041008DF842408DF8437010A802F032FF6B
:100A300001224FF49061304600F0E8F80121304681
:100A4000FFF740FF01213046FFF732FF0121284622
:100A5000FFF72EFF304600F06EF9304600F09FF8A9
:100A60000028FAD1304600F075F9304600F082F8DF
:100A70000028FAD1284600F05EF9284600F08FF8E9
:100A80000028FAD1284600F065F9284600F072F8EF
:100A90000028FAD10121084603F01AFA154D28461C
:100AA00000F0A6FD684600F04EFE0F4801A94C304C
:100AB0000090114881E811018020CDE904404000F8
:100AC000069080000790202008904FF44050CDE918
:100AD00009046946284600F019FE0121284600F065
:100AE0007BFD12B0BDE8F0810024014000280140E8
:100AF000002C014008000240A00200200D4910B562
:100B0000884202D1012144150AE00B49884202D1F2
:100B10000121041504E0094988420AD10121CC03CE
:100B2000204603F005FA2046BDE81040002103F0FE
:100B3000FFB910BD0024014000280140003C0140E5
:100B40000029816802D041F4801101E021F4801174
:100B5000816070470029816802D041F4004101E0C2
:100B600021F4004181607047826822F4E0420A4328
:100B700082607047014600208968490700D501203E
:100B8000704710B50246002054680B0AC9B20C40E9
:100B90001168194202D0002C00D0012010BD01467E
:100BA00000208968090700D50120704738B5012168
:100BB0001C2003F0B1F9FF20ADF8000000248DF8EF
:100BC000034003258DF8025069460D4801F02EFBC5
:100BD0000120ADF800008DF803408DF80250694601
:100BE000084801F023FB2320ADF800008DF80340F6
:100BF0008DF802506946044801F018FB38BD00002A
:100C000000080140000C014000100140002A426829
:100C1000C9B201D00A4300E08A4342607047000035
:100C200010B542680E4B0C791A400B6842EA042258
:100C30001343436083680B4A1340D1E902422243C5
:100C40004C7943EA44031A438260C26A097C22F465
:100C50007002491EC9B242EA0151C16210BD0000D2
:100C6000FFFEF0FFFDF7F1FF70B5072409290AD94F
:100C7000C568A1F10A0606EB4606B440A543B34099
:100C80001D43C56007E0056901EB4106B440A5437B
:100C9000B3401D430561836BC3F30154121B921CC7
:100CA00002EB82041F22A2409343A1400B438363C3
:100CB00070BD826B491E22F4401242EA01518163E9
:100CC000704770B5072409290AD9C568A1F10A0639
:100CD00006EB4606B440A543B3401D43C56007E09C
:100CE000056901EB4106B440A543B3401D430561CE
:100CF0001F23072A09D2446B521E02EB8202934043
:100D00009C4391400C43446370BD0D2A09D2046B8F
:100D1000D21F02EB820293409C4391400C43046338
:100D200070BDC46A0D3A02EB820293409C4391402D
:100D30000C43C46270BD816841F008018160704756
:100D40000029816802D041F4A00101E021F4A00152
:100D500081607047816841F0040181607047002123
:100D60000160017141718160C160012101747047AE
:100D700070B51E4C214694F83800B1F84250062850
:100D80001ED9B4F84A10B4F84C00A1EB000202F1ED
:100D90000902122A04D8FFF753FB0022144B0AE081
:100DA000884204D2FFF74CFB0022124B03E0FFF70E
:100DB00047FB0022104BFFF72CFAFFF786FB09E0F8
:100DC00005D12846FFF73CFB0C4A0D4BF3E70D49D4
:100DD00051F82000C5EB45116063B0EB410F03D91A
:100DE000C5EB45104000606370BD00003404002076
:100DF00000003440000033400000354067666666FE
:100E000066E64B40EC88000810B50C4C2078400793
:100E100013D5FFF7ADFF0A49A08E08800848303887
:100E2000018821F010010180001F018841F01001AC
:100E30000180207820F00400207010BD34040020D0
:100E400040040040F0B41448144B154A816804462D
:100E50001B782468526CCF0541F0080521F0080684
:100E60004FEA047413D5002C07DB090712D4002BBA
:100E700010D1142A0EDA856006E009070AD5002B86
:100E800008D1142A06DA8660F0BC05F081BD002C7A
:100E9000F3DAEAE7F0BC704790020020E706002092
:100EA0003401002070B506464089204B204C4FF499
:100EB0008071002580B362887AB1012A0CD1E18863
:100EC000491C89B2E1803289914205D36580E58071
:100ED000FF2801D0401E708170BD7088228890422A
:100EE00001D9012200E00022184601F028FA70889A
:100EF000B18801442088401C80B220808142EBD818
:100F00002580A088401C80B2A080F1888842E3D36D
:100F100001206080A58070BDFFE70022184601F027
:100F20000EFAA580E58025806580F4E7000C01407D
:100F3000A4050020FEE70000FCB505464FF6FF764D
:100F400000200C46ADF8006048F205078DF804005B
:100F500020E000BF15F8010B8DF8040001A9084638
:100F600002F0FCF8BDF800009DF8041080EA0120B2
:100F7000ADF800005FF00000BDF800100A0402D5D3
:100F800087EA410101E006EA4101401CADF800108A
:100F90000828F1DB641EDDD26946084602F0C8F875
:100FA000BDF80000FCBD00000246002004E000BFC8
:100FB00012F8013B1844C0B2491EF9D27047000034
:100FC00070B5144A85B01088002413490194009428
:100FD000039420460494138807E00D8B009E35444B
:100FE0000095CD8B019E3544019515889D42F4D026
:100FF000401CC0B28028EED30098411107484180C0
:10100000848001984111064881830183818205B063
:1010100070BD0000F006002090020020BE050020F8
:10102000AC04002030B50E4902880A800C4A43887F
:10103000083A13800B1F808818802024151F2C80ED
:101040000020401C80B27328FBD341F211100880AD
:1010500044F64800108047F2480018802C8030BDCC
:10106000202C0140114944F648000880091D46F62D
:1010700048000880091D41F2111008800B48001F2C
:10108000018841F02001018009480021A0F8641086
:10109000A0F86210A0F86010A0F85E10A0F85C1034
:1010A000A0F85A100348418181827047182C0140F2
:1010B000900200205C000020F0B54D4B4D4800210F
:1010C000DA7A0778802A27F001057CD31C684A4B1E
:1010D00002F01F0253F82220484B14421A6802D033
:1010E00042F0200201E022F02002454C1A60454EF9
:1010F00094F800C0444CBCF1020FB4F904403FD155
:10110000B3F808C0CCF3C00ECCF3002CE64537D0C2
:101110003A4D2C3D95F802C0BCF1000F04D0BCF153
:10112000010F0FD0A9702FE05FEA025C2CD55FEAB7
:10113000826C29D44FF0010C85F802C027F0040519
:10114000057021E05FEA025C1ED45FEA826C1BD569
:101150005FEA477C11D447F004070770B0F802C07B
:10116000BCF1000F03D0418027F0010704E0448068
:10117000002C02DD47F0010707700227AF7003E083
:1011800005704180318041811C4DC78895F84650DB
:101190000FB9002C15DC077BAF4212D1B0F90270F9
:1011A00007F26667BC420CDC184FBF895FEA477CD8
:1011B00007D45FEA877C04D45FEA427C01D5FF074D
:1011C0000BD0077800E00FE05FEAC77C05D027F07E
:1011D00001070770418031804181C4800573500947
:1011E00060F3CB221A60F0BD057041804181F0BDF3
:1011F000C4050020F80800204C8D00089002002053
:10120000E706002008010020BE050020000A00209B
:101210002DE9F04796B000240C940D940E940F9491
:1012200072B69048816941F400718161816941F42D
:10123000806181614FF4004002F040FE8A4D002140
:101240002846FFF73FFB00212846FFF731FB874E7A
:1012500000213046FFF72CFB854F0021384600F077
:10126000BBF901204FF47041401C8842FCD3284652
:10127000FFF744FCB1463046FFF740FC384600F02B
:10128000B7F94FF46020CDE912048DF845400120F4
:101290004FF004088DF8440010948DF8508010A988
:1012A0002846FFF7BDFC01231A4605212846FFF713
:1012B00008FD0123022206212846FFF702FD012333
:1012C000032207212846FFF7FCFC012304220F21FB
:1012D0002846FFF7F6FC384600F08AF9684600F029
:1012E00032FA6148634E4C300090CDF80C80CDE965
:1012F00001648020CDE90440400006908000079002
:10130000202008904FF44050CDE909046946384642
:1013100000F0FCF901212846FFF7D4FA01213846F4
:1013200000F05AF901212846FFF7C2FA47F230517E
:1013300015941598401C15908842FAD3012128462F
:10134000FFF7FEFCADF82C40A04640F2DC5A4FF40B
:10135000007420E05046CDF854801599491C159131
:101360008142FAD330880D9908440D9070880E9907
:1013700008440E90B0880F9908440F90F0880C999B
:1013800008440C9001212846FFF7DAFCBDF82C0038
:10139000401CADF82C00BDF82C00A042DAD30D980B
:1013A000354A40F3CF1633480A3006830E9941F38D
:1013B000CF1444830F9941F3CF1383830C9941F3E6
:1013C000CF1CA0F804C0ACF5C05C40F2C371ACF512
:1013D0009B7C8C450ED2A6F5C856363E8E4209D26D
:1013E000A4F5C854363C8C4204D2A3F5C853363B0E
:1013F0008B4203D3D18841F48041D180D188490404
:1014000007D41E49028B21F85C2F428B4A80808BC7
:10141000888000212846FFF755FA0021384600F061
:10142000DBF800212846FFF743FA00214C464846E6
:10143000FFF73EFA0220C102401C8842FCD3284636
:10144000FFF75CFB2046FFF759FB384600F0D0F869
:10145000FFF742FA0A493C20087062B616B0BDE8B0
:10146000F0870000001002400024014000280140E5
:10147000080002400A050020000A0020540C002049
:10148000E4060020F0B5384B394C93F85250374BF6
:10149000042D5B6C1DD0256840F22D465D1B6560F8
:1014A00043F6FB25B3F5FA5F33DDB3F5FA4F30DCD5
:1014B00041F6AD17A3F5FA535F4306EBA7364FF499
:1014C000B5777B4305EBA31375105B10C4E9065396
:1014D00021E043F6D017102641F26205BB4218DB2B
:1014E00044F25067BB420EDAA3F5645345F24C67F1
:1014F000D03B5F4306EBA736A66140F624767343E4
:1015000005EB232303E042F24713A361194BE36188
:1015100001E0C4E90665A3695360E569401AD56036
:1015200010604543107C0541106A29181162D0698A
:10153000814200DD1062116A9069814201DB084638
:1015400000E01062206211684B43117A0B410841A0
:101550001918B2F91400884204DBB2F9120088426B
:1015600000DC08B2F0BD00005C0000203401002067
:101570000C01002085EB010010B54FF4005420460B
:1015800000F0ACF8002813D00A49087840F00800B1
:101590000870204600F014F80021074800F01CF8FD
:1015A0000648C17E012903D10021C17601210177BE
:1015B00010BD00005E06002044000240F80A002032
:1015C000C10002D50249086070470249486070476F
:1015D00004040240000002400029016802D041F0EA
:1015E000010102E04FF6FE721140016070470000F9
:1015F00001684FF6FE7211400160002101604160F8
:101600008160C1603149314A0839904203D148684C
:1016100040F00F0006E02D4A1432904204D1486891
:1016200040F0F00048607047284A2832904203D1C9
:10163000486840F47060F5E7244A3C32904203D198
:10164000486840F47040EDE7204A5032904203D1A0
:10165000486840F47020E5E71C4A6432904203D1A8
:10166000486840F47000DDE7184A7832904203D1B0
:10167000486840F07060D5E7154A111F904203D1C9
:10168000086840F00F0006E0114A1432904204D17D
:10169000086840F0F000086070470D4A2832904218
:1016A00003D1086840F47060F5E7094A3C32904283
:1016B00003D1086840F47040EDE7054A503290428B
:1016C000EAD1086840F47020E5E700000800024015
:1016D00008040240406880B27047000001460020C4
:1016E000CA0001D5034A00E0034A12680A4200D04A
:1016F000012070470004024000000240002A0268F6
:1017000001D00A4300E08A430260704730B50368A5
:1017100047F6F07293430C6A8A682243D1E9044584
:101720002C4322438C692243CC6922434C6A2243D6
:101730008C6A22431A430260CA6842600A68826067
:101740004968C16030BD0021016041608160C160B5
:10175000016141618161C1610162416281627047E1
:1017600010B5114C8CB000212046FFF735FF204604
:10177000FFF73EFF0D4800900D480021CDE9010123
:101780006420CDE903018020CDE90501079108918E
:1017900009910A9169462046FFF7B8FF01212046CA
:1017A000FFF71AFF0CB010BD58000240043801408A
:1017B0007C07002010B501218CB0084602F088FBA0
:1017C0001E4C00212046FFF707FF2046FFF710FFC1
:1017D0001B4800901B48019000211020CDE9020118
:1017E0008020CDE9041006910791089109910A9192
:1017F00069462046FFF78AFF012202212046FFF7B3
:101800007DFF01218DF82F1004208DF82D008DF81B
:101810002E100E208DF82C000BA802F03BF80F20A4
:101820008DF82C000BA802F035F801212046FFF7B7
:10183000D3FEFFF795FF0CB010BD0000440002403E
:10184000043801401807002030B540F6AA21204A8C
:10185000C184838B1488E31A9BB20F2B10D3128898
:101860008283037E002253B11A4BB3F90A30052B51
:1018700005DB194B1B78022B03D0002B00D182848F
:1018800030BD164B40F68B255B6CA3F22D14AC4299
:101890000FD2428B521C92B24283642AF0D364224C
:1018A0004283B0F924208A4201DA02EB21118184BB
:1018B00030BD41F29414A342FADBB0F92430002B7E
:1018C00002DDA3EB211100E000218184428330BDC1
:1018D000F00600205C000020E70600203401002014
:1018E00010B50446B0F9020043F69911484381133C
:1018F000E06840F26662504301EBA030E060B4F96A
:10190000001043F6991251438A13216940F266632D
:10191000594302EBA131216104F0A8FC6061A18868
:1019200040F6AB2208444010A0F515415539E0625D
:10193000914205D9A0F5F851FF39521C91421DD2B0
:1019400049F25451884202DDA0F5204002E0A0F5A2
:10195000F850FF38206300EB400040F34F00208533
:10196000B4F924104A42904201DA104602E088425B
:1019700000DD0846E083228461848AE0A0F5FE420F
:10198000FF3A41F255518A4214D8A2F6AA202063A8
:1019900000EB400040F34F002085B4F92420514271
:1019A000E183884201DA084602E0904200DD1046F9
:1019B000404250E0A0F5D442AA3A8A4215D2A2F69B
:1019C000AA20206300EB400040F34F012185B4F9C9
:1019D00024004242E2832084914201DA104602E070
:1019E000814200DC0846608453E0A0F5AA42543AE4
:1019F00041F256539A4215D2A2F6AB20206300EB77
:101A0000400040F34F002085B4F924104A42904230
:101A100001DA104602E0884200DD08464042E083D9
:101A2000218419E0A0F5804241F254539A4215D224
:101A3000A2F6AA20206300EB400040F34F0121856D
:101A4000B4F92400E0834242914201DA104602E0F8
:101A5000814200DC0846208462841AE0A0F5285206
:101A6000AB3A8A4215D2A2F6AA20206300EB4000CE
:101A700040F34F012185B4F92400E08342422284DF
:101A8000914201DA104602E0814200DC0846404201
:101A9000A9E7B4F91E006FF4BF7148438013E080DA
:101AA000B4F92000484380132081B4F92200484350
:101AB0008013608110BD01210176704770470000DE
:101AC0001548164A4FF480410078042821D002F1CD
:101AD0003C03D08A9B88C01A00B22F2801DD001178
:101AE00008E0002801DD002007E00D4B984201DAF4
:101AF000184602E0402800DD40209389184400B2D7
:101B0000884203DC40F26661884200DA0846908130
:101B10007047918170470000E7060020AC04002068
:101B2000C0FEFFFF38B54B484B4902880B889A1A14
:101B300092B20F2A71D30988484C01804FF0FF01FF
:101B4000E2884FF47A7355044FF4967002D516224A
:101B5000009103E0950403D515220091014670E041
:101B6000D50402D514220091F8E7150502D51322F9
:101B70000091F3E7550502D512220091EEE7950595
:101B800002D511220091E9E7D50502D51022009176
:101B9000E4E7150602D50F220091DFE7550602D5CE
:101BA0000E220091DAE7950602D50D220091D5E7C5
:101BB000D50602D50C220091D0E7150702D50B22DD
:101BC0000091CBE7550702D50A220091C6E7950799
:101BD00002D509220091C1E7D20702D00822009164
:101BE000BCE72289550702D507220091B6E7950781
:101BF00002D506220091B1E7D20702D0052200915A
:101C0000ACE7A27AD20702D004220091A6E7A2890B
:101C1000D40603D503220091A0E719E0140702D5EA
:101C2000022200919AE7540703D4940701D4D20703
:101C300002D00122009191E70020034602460146AE
:101C4000009002F00BFEBDE838400248FFF72AB9C9
:101C500038BD0000F4090020F0060020000A002032
:101C6000F0B55948594982880B889A1A92B29C2A31
:101C700064D30988818056490A880146002A0B7876
:101C800043F0020156D11646524A1C071568024617
:101C9000127822F0020274D54F4C0746E4887F7810
:101CA0005FEA845C02D547F0010701E027F00107F5
:101CB0004770A704477802D547F0020701E027F0F4
:101CC00002074770670401D4E70703D0477847F05D
:101CD00008074770640603D5447844F0040404E020
:101CE0001C0603D4447824F004044470EC0450D45B
:101CF000354C9A07247824F0100423D4324D4278CE
:101D00002F7A2D78012A45F0100514D0022A16D01A
:101D10002D4C042AA47804F1010C0CF0FF0C13D014
:101D2000072A25D0032A23D0052A21D0062A1FD02E
:101D300021F0100142E0B90702E00570F0BD39075B
:101D40000029FADB0470F0BDFA0601D41A060AD5A0
:101D50000170022C04D280F802C0BCF1020FF2D351
:101D600041F080012AE021F0100101708670F0BD81
:101D7000877A7F06F7D5032C04D8017080F802C05B
:101D8000F0BD0FE05107D8D51906D6D443F0800135
:101D900014E002704178CB0701D18907F0D522F019
:101DA00010010BE0E9040BD49907E9D4818AC82912
:101DB00002D2491C8182E3E743F00A010170DFE7A8
:101DC00002708682DCE70000C8060020F0060020D2
:101DD000F206002090020020000A0020094944F683
:101DE00048000880091D46F648000880091D41F694
:101DF000CC4008800348001F018841F02001018089
:101E000070470000182C0140084946F66800088019
:101E1000091D0880091D41F2555008800348001F24
:101E2000018841F02001018070470000182C01401A
:101E300010B5C28800210AB1032206E002890AB166
:101E4000022202E0428912B10122027000E0017018
:101E500004784FF4804344F6206244B1012C06D04C
:101E6000022C07D0032C01D14180818010BD43801A
:101E7000828010BD41F23331418040F6B731F4E742
:101E800030B5B1F86A5000231A240D22854202DCD5
:101E9000B1F9680030BD4D88854202DBB1F9000020
:101EA00030BD01EB82056D88854201DD144601E0FD
:101EB00013DA134604EB03024FEA52029A42F0D1BE
:101EC00001EB830231F8231054889288521A001BC8
:101ED000424301EB622000B230BD31F9220030BD37
:101EE00030B5CD8D00230B240522854202DCB1F9EB
:101EF0002C0030BD4D88854202DBB1F9000030BDB9
:101F000001EB82056D88854201DD144601E013DA9C
:101F1000134604EB03024FEA52029A42F0D101EB5E
:101F2000830231F8231054889288521A001B4243CE
:101F300001EBA22000B230BD31F9220030BD00001B
:101F4000054920B1086940F08000086170470348E6
:101F500048600348486070470020024023016745FD
:101F6000AB89EFCD06494FF47A70CA68D20705D025
:101F7000401E0004000CF8D1FF207047002070477D
:101F80000020024012480321A0F1480280F83210DC
:101F90000021D1800F4A11860F4A1186D162D18368
:101FA0001184518441620D498A6CB2F5206F01DBC6
:101FB000A3224262897A11B1416A49424162816A2F
:101FC00041F39101416288030549086270470000AE
:101FD0005C00002090020020140500203401002045
:101FE0005C080020F0B53B4988894A89801A80B294
:101FF0000F2866D388894881CA8937480B3A272A2F
:1020000026D28A7822BB8268364B42F48072826084
:10201000324A354C354D12785607314A0AD4344E7F
:1020200036881680334A12881A80334A12882280F2
:10203000324A09E0324E36881680324A12881A80B7
:10204000314A12882280314A12882A8001228A70FD
:102050002F4B304D19469A7F0968802A32D302F0FF
:102060001F0255F8222011422CD0826822F48012DF
:10207000184E8260123614461215B778521C62F35D
:102080008617254AB77093F816C01778BCF1800FF1
:1020900027F0020608D30CF01F0C55F82CC011EAEB
:1020A0000C0F01D147F0020616701A7E802A0DD35C
:1020B00002F01F0255F82220114207D144F40021FA
:1020C0008160F0BD826842F48012D1E724F40021DF
:1020D000F6E70000E4060020900200203401002012
:1020E000A4040020A6040020A8040020AA040020C4
:1020F0009404002096040020980400209A040020F4
:102100009C0400209E040020A0040020A2040020C3
:10211000C40500204C8D0008AC04002070B5204898
:1021200081890289891A89B20F292FD38189018176
:102130001C4B1D4819465D7A06681C4C096846F020
:102140000402802D07D305F01F0554F825502942BD
:1021500001D126F0040202609A7B802A17D302F094
:102160001F0254F82220114211D1026822F002020B
:102170000260DA7A802A0ED302F01F0254F822207D
:10218000114208D1016821F00801016070BD0268A8
:1021900042F00202ECE7016841F00801F5E70000B7
:1021A000E4060020C4050020900200204C8D0008A9
:1021B000F0B51D4C1B4A4FF0010C94F83B5094F8BD
:1021C0000AE0144692F83C3094F838402B43651CE2
:1021D000EEB2154D95F83D700025BEF1FF0F0AD007
:1021E000BEF1000F06D18B4213D155700C2C01D2D9
:1021F00082F83860F0BD834202D182F801C0F5E771
:102200008B42F7D15570B80709E000BF82F838500B
:10221000F0BD8342FCD1F84382F801C0800700285A
:10222000F4D0F0BD3404002034010020F0B5CA78A9
:10223000002502F00F03D20601D58A7813430A78ED
:102240004FF00F0E12F0FF0F4FF001021CD0046888
:102250000F8802FA05F63740B74211D14FEA850CD4
:102260000EFA0CF724EA070703FA0CF43C43CF7884
:10227000282F02D0482F02D002E0466100E006611C
:102280006D1C082DE4D304600C88FF2C1ED9446813
:102290005FF0000606F1080702FA07F50F882F40E5
:1022A000AF420FD14FEA860C0EFA0CF7BC4303FA8B
:1022B0000CF73C43CF78282F00D14561CF78482FC9
:1022C00000D10561761C082EE4D34460F0BD000007
:1022D000F0B5144C002801DAE36900E06368420DB0
:1022E000120185B2C0F301579540C0F30346032F96
:1022F00005D0C2020AD50322B240934307E023F07F
:102300007062636823F07063636002E0AB4343F084
:10231000706201B12A43002801DAE261F0BD626017
:10232000F0BD0000000001400246002092680A4211
:1023300000D00120704741617047016170470AB1C8
:1023400001617047416170470F4A104B92F8381095
:102350005B5C834201D1012004E00D4B5B5C834256
:1023600003D1002082F83A0070470A4B5B5C83423D
:1023700001D18120F6E7084B595C814201D18020D0
:10238000F0E70320EEE70000340100200C91000884
:102390001E91000812910008249100080A4810B507
:1023A00001784FF000024C0708494FF0FF0389689D
:1023B0004FEA017105D5002901DA827210BD8372DE
:1023C00010BD0029FBDBF8E734010020900200205B
:1023D000F0B5194E194C0022E31CA6F1060CB75CAF
:1023E000A518ED78FF5C0D430F43BD421FD01CF8CC
:1023F0000270FF5C0F43BD4219D015460023A6189A
:10240000F6780E43C6545B1C1CF80220DBB2062B88
:10241000F5D3C17881700179C17000214218491C3F
:1024200015711CF80550C9B20629F7D3F0BD521C2E
:10243000D2B2032AD3D3F0BDDE88000834040020D2
:1024400010B502460021064B06205C1864789442C1
:1024500000D10846491CC9B20629F6D310BD0000B8
:1024600034010020214810B590F867100022204860
:10247000012936D11F49898899BB1F491E4B4C6CD5
:1024800040F6B831B3F86E308C4227DD1B4909782D
:1024900021BB90F82711491CC9B280F82711C8291F
:1024A0001CD380F827210146D0F82C4191F828113F
:1024B000A34203DD052908D2491C01E041B1491EB0
:1024C00080F82811C9B2052902D3012180F826110C
:1024D000191B074C2C3C6162C0F82C31B3F5FA6F24
:1024E00003D280F8262180F8282110BD540C00204A
:1024F00090020020BE05002034010020E7060020E5
:102500004FF4C0428260002141620E22828141F27A
:1025100062020261082282824FF46042C282018319
:102520004FF07842C0E9072140F6C411018070479E
:10253000B0F90010B0F90220891A41600269037DE8
:102540004A431A41436A13444362026A934200DDDC
:102550004262436AC269934200DA42628268436A15
:102560004A43017B0A410B41D118B0F918208A4235
:1025700001DA10467047B0F916008842FADC08B25A
:102580007047000010B514481449B0F88C200B882F
:102590009A1A92B2B2F5437F1DD90988A0F88C101F
:1025A000B0F88A1020F8581F002242860C480D4CC3
:1025B000C2888280C180C38983812489891AA4B298
:1025C000C4818160E11A0161074A818AC182928ACD
:1025D0008282511A816110BD34010020F006002072
:1025E0001C0C0020140500205C00002009480A494A
:1025F000B0F8AA200B889A1A92B241F684639A42E4
:1026000006D3098820F8AA1F4188818000214180D3
:102610007047000034010020F00600200D480178CA
:10262000C90702D00C49098801E04FF6FA71C1656B
:10263000094901201039088007482438018841F0F1
:102640000101018004481838018821F01801018037
:102650007047000034010020240400400A49D1F8EA
:10266000902012B1521EC1F8902031F88A2F521CCE
:1026700021F81A294A6A521C4A628A8F521C8A8798
:1026800001F8380C70470000340100201CB52D48BB
:1026900090F83B3090F83C20934252D000248DF8C3
:1026A000044053408DF800309DF800300122012B8A
:1026B00008D09DF80030022B09D09DF80030042B83
:1026C0000AD00DE01F498DF80420443108E01D496F
:1026D0008DF80420463103E01A498DF80420483172
:1026E0009DF80420012A2CD190F83D309DF800403F
:1026F000154AA34217D090F83E309DF8004023427F
:1027000008D0B0F84C30A0F84A300B881488E31A8F
:10271000A0F84C3090F838302BB1B0F84030148825
:10272000E31AA0F8423012880A80A0F8402010F87E
:102730003E1F9DF80020114300F801199DF800107C
:1027400001701CBD34040020F006002070B5344D2B
:1027500040212846FFF7E8FD840080212846FFF746
:10276000E3FD44EA4004A9152846FFF7DDFD0443D4
:10277000E1B22C4C94F870508D4250D04D4084F80A
:102780007010012D03D0022D01D0042D47D194F8F3
:102790007400A84384F8740094F87320AA420FD000
:1027A00084F8735094F8722001238B401A4207D1A9
:1027B0001A4384F8722094F87110491C84F871103F
:1027C00094F87110042928D330B1012811D00228BF
:1027D0000FD004280DD012E01348C18821F0400129
:1027E000C1802078002184F83B1020F06000207028
:1027F00005E0217841F02001217084F83B000B496D
:1028000094F83B0091F82720904204D081F82700EB
:1028100007492020087000F00DF884F84C5070BD76
:102820000010014034010020000A0020540C002058
:10283000E406002070B50D4D40212846FFF774FDD9
:10284000840080212846FFF76FFD44EA4004A91563
:102850002846FFF769FD04430548072100F8704F3B
:102860000171002141708170C17070BD0010014084
:102870003401002070B5344890F83A10CA439207EA
:1028800061D001F0030280F8392090F83D305B06FA
:102890001B0E80F83D30012A01D0812A02D15B1C39
:1028A00080F83D300278D2074DD0DBB203F0010250
:1028B000C3F34004A24246D1B0F84E400025641C48
:1028C000A0F84E40204CA0F8505090F83E60A47AFA
:1028D000B24202D080F83E200DE0A607B6EB837F1F
:1028E00002D080F83F5006E090F83F30642B02D2CF
:1028F0005B1C80F83F3090F84030642B0CD25B1C9E
:10290000DBB280F84030022B06D204F00103934280
:1029100002D1022280F84020012901D0002912D1E1
:1029200090F83820C16D00EB820291610163D0E91B
:1029300006121144D0E908231A441144826A114452
:10294000C26A1144416370BD34010020FEE70000FB
:102950002DE9F04F00BF00209E4E9F4AA6F5127150
:10296000A6F5BE79A6F1440B06F1440E804601F5AA
:10297000E074A1F1780301F5457A1D5C15F0C007FC
:1029800006D0402F51D0C02F77D0802F76D004E1D1
:1029900015F01F0504D0154440F080072F7201E0A8
:1029A00082F80880012826D0022824D0032822D0CB
:1029B000042820D008281ED010281CD0874D55F898
:1029C00020C0DCF8005054F820703D40CCF8005096
:1029D000824D55F820C0DCF8005056F820703D4379
:1029E000CCF800501D5CAD0659F820502F6813D567
:1029F0003AF810C03EE051F820502F6854F820C03B
:102A000007EA0C072F6051F820502F6856F820C0B5
:102A100047EA0C072F60E5E7DFF8B8C10CF1F00CCE
:102A20005CF820C007EA0C077EE015F01F0504D013
:102A3000154440F080072F7201E082F808800128D9
:102A40001DD002281BD0032819D0042817D008282D
:102A500015D0102813D0614D55F820502F6854F828
:102A600020C007EA0C072F605C4D55F820502F68F6
:102A70005BF820C047EA0C0756E00BE056E051F83F
:102A800020502F6854F820C007EA0C072F6051F837
:102A90002050ECE715F01F0505D0154440F08007E5
:102AA00085F8217001E082F82180012825D00228D4
:102AB00023D0032821D004281FD008281DD0102897
:102AC0001BD0464D55F820C0DCF8005054F820705B
:102AD0003D40CCF80050414D55F820C0DCF8005086
:102AE0005EF820703D43CCF800501D5CAD0615D556
:102AF0003A4D3AF81070CC3514E051F820502F6858
:102B000054F820C007EA0C072F6051F820502F68B6
:102B10005EF820C047EA0C072F60E6E72D4D3AF833
:102B20001070E03D55F820502F6036E015F01F057D
:102B300005D0154440F0800785F8217001E082F847
:102B40002180012830D002282ED003282CD0042840
:102B50002AD0082828D0102826D0204D55F820C08B
:102B6000DCF8005054F820703D40CCF800501B4D6C
:102B700055F820C0DCF80050164F883757F8207001
:102B80003D43CCF800501D5CAD06B1D4114F3AF86E
:102B90001050E03F57F820703D60401CC0B2112833
:102BA000FFF4EBAEBDE8F08F51F820502F6854F8D9
:102BB00020C007EA0C072F6051F820502F68DFF87B
:102BC00014C00CF1880C5CF820C047EA0C072F6099
:102BD000D9E70000D88F0008C4050020D48D000874
:102BE0004FF40771C1824FF45861018340F61451CC
:102BF00081837047F0B5C48AB0F900608681B0F96E
:102C00000250C581B0F9043002270021012203825D
:102C1000AB4204DBB54202DDC78042810CE0B34227
:102C200004DBAE4202DDC78041811CE09D4205DB32
:102C3000B34203DDC2804781018115E0B54204DB68
:102C40009E4202DDC280418105E0AE4205DB9D422D
:102C500003DDC1804281078106E09E4204DBAB4276
:102C600002DDC18047810281C388458900EB4307AB
:102C700000EB4505BB89AE899B1B0FFA83FEA0F8CC
:102C800012E00689AB8900EB460CBCF80CC0A3EB44
:102C90000C038382B0F91830B7F90CC0A3EB0C0C0D
:102CA000B4EB4C0F04DA80F82010A3F1A10113E07B
:102CB000A64503DD80F82010B9890BE026B1012E6E
:102CC00004D0022E10D004E0062100E0052180F897
:102CD0002010A989091B6D31418309B2B1F5586FE4
:102CE00004DB5B1E438304E00421F0E7002900DCE1
:102CF0004283418B8183F0BD0B49002288760A62B2
:102D0000CA614A62094A32F9103002EB40028B6212
:102D1000B2F90220CA62064A32F810000882A1F80D
:102D20006000A1F862007047E401002036910008BD
:102D30002A9100082DE9F05FEF48F04982880B885E
:102D40009A1A92B20F2A44D309888180EC498246AC
:102D500001270888EB4CEC4E002578B3401E088014
:102D6000E573EA49A5622068B1F90210430742F60B
:102D7000AA2218D4F38843F40053F380E34B1B7862
:102D80009B0709D5A36823F08003A360A4F87C50B7
:102D900084F87E5084F87F50C30404D484F8F07023
:102DA000C4F8EC5003E084F8F050430707D4914294
:102DB00005DB84F8F470A4F8F25004E010E084F825
:102DC000F450430703D4914201DBC00703D084F8D9
:102DD0001151BDE8F09F84F81171A4F81251F8E781
:102DE000B4F8180143F69821884202D2401CA4F896
:102DF000180101F049FDDFF81883DFF8FCB298F8FC
:102E00005000ABF1180B10B1FEF756F905E09BF836
:102E1000001021F001018BF8001098F8630010B148
:102E2000FEF710F808E0A068C10502D520F0080000
:102E300001E040F00800A060FFF714FB00F0A4F9E7
:102E4000B44841F26801436C4FF400608B4201DBEF
:102E5000B14904E0B3F57A6F02DAAF49091D0860A1
:102E600098F85100C646C107DFF89882AB48DFF8F2
:102E7000B092A8F12C0839D0817B802932D32178F7
:102E800089072FD4E27B88F80520A04A414692F8B2
:102E900000C02CF0020C82F800C0ABF80250CBF856
:102EA00014509BF800C02CF0010C8BF800C0B279D4
:102EB000520612D44A8941F2883C624503D2521C20
:102EC000A8F80A2012E040F63C70834201DD0020A1
:102ED000DEE0042088F80370DAE0CD700020A8F866
:102EE0000A50D5E088F80350A8F80A50A1680A05EE
:102EF00001D50820CCE09EF83FE05FEACE7240D0DA
:102F0000E27B88F80520437A802B59D323785B072E
:102F100030D4F3889B0403D521F02000A06030E07A
:102F2000ABF80250CBF814509BF800C041F02001E0
:102F30002CF0010C8BF800C0A160C17D802909D361
:102F400001F07F0300684FF00041D940084201D1F1
:102F5000277100E025712079C00702D15FEA8E70E9
:102F600005D50320032A01D088F8087090E00020DE
:102F7000A5628DE021F02000A060F08820F40050D0
:102F8000F08094F8260101281FD094F8462043F2DF
:102F900033304FF48047D2B143F69911012A2CD037
:102FA00099F800205F48C2F38102012A28D0022A42
:102FB00026D090F85200A4F81471042831D025E0EE
:102FC000206840F004002060A6E7092060E099F83E
:102FD0000010C1F38101012909D002290AD042F66B
:102FE000B86100BFA4F81411A4F8440010E042F640
:102FF000CC41F7E742F26661F4E7A4F8140110E06F
:10300000A4F8147190F8520004280AD0A4F844706F
:10301000FEF752F89BF80010C90705D0BBF8021064
:1030200004E0A4F84410F3E738488188AAF81210A5
:1030300008B2B4F944104843C0F38F314046A8F8B1
:103040001210B94200D9478237490978C90605D517
:10305000428A41F233318A4200D241822189C1F34E
:10306000C002C1F300218A4205D1428A40F6CC4118
:103070008A4200D94182B17AC90700D04582B8F8A6
:103080001200A06200287FF722AF284805700220B6
:103090009AF81A1099B9022824D080B11D490B78EA
:1030A0009D0608D5B5796D0605D51F4D2D78ED091E
:1030B00065F386130B70F18821F40A61F1801549DC
:1030C000496C4E290ADBF1880B0607D521F08001F7
:1030D000F1800E490B7823F002030B708AF81A0076
:1030E000E07376E6B9F83830002BD7D143F6982351
:1030F000A9F83830D2E7000010090020F0060020BF
:10310000F206002090020020000A0020BE050020E8
:10311000540C002034010020100C0140C405002094
:10312000AC0400205C000020C8060020040700203A
:1031300070B500230C8863F30F02012505FA03F62E
:10314000344206D0C3F10F0605FA06F1114361F3CC
:103150000F025B1C102BF1DB028070BD70B50023E9
:103160000C7863F30702012505FA03F6344206D012
:10317000C3F1070605FA06F1114361F307025B1C70
:10318000082BF1DB027070BDF0B51F4890F8663077
:103190001E48012B816821F4006232D11C4BDE886D
:1031A00074062ED41B4D0F054FF00004B5F90250E4
:1031B0001ED4194A526C642A11DC40F638629542DA
:1031C0000DDAB2040BD4027852070ED4B0F8D42032
:1031D00040F6B835AA4203D2521CA0F8D420F0BD64
:1031E00041F4006181605C81F0BDA0F8D440F0BD85
:1031F00041F2CD018D42FADD997AC907F7D182609B
:10320000F3E78260F0BD0000540C00209002002023
:10321000000A0020BE05002034010020F0B5364D24
:10322000364F044695F83B0097F83B102378084347
:10323000EE1C6278834205D1E0781146FEF7B8FFB4
:10324000207908E094F802C084450CD1E17810465A
:10325000FEF7AEFFE07905F82F0F2878805D6870E3
:10326000287BE877F0BD82421DD161461846FEF703
:103270009FFF95F84E1095F83B00814207D1B97A2F
:1032800009B1A17900E0617985F82F101EE0697815
:10329000012901D0A17922E0617927E0297841F064
:1032A0000401297012E0E1788142DBD119466046C1
:1032B000FEF77EFF95F84E1095F83B0081420AD14B
:1032C000B97A09B1617ADFE7217ADDE715F82F1FB6
:1032D000895D6970C5E76978012906D0617A85F84A
:1032E0002F10B97A0029F1D1D8E7217A85F82F106B
:1032F000B97A0029EAD0D1E7340400203401002053
:103300000B48017821F0020100F8381B002100F879
:1033100018194177817733218185418508214184BE
:10332000012100F81F1C034880F839107047000085
:1033300034040020340100200D4900B50B4851F839
:10334000012F40F8032F8988818008480121093026
:10335000FFF73EF8054802211330FFF739F803481C
:1033600004211D305DF804EBFFF732B8340400206F
:1033700034010020094944F648000880091D46F63A
:1033800048000880091D41F2111008800348001F01
:10339000018841F02001018070470000182C014095
:1033A0002DE9F047664C674B0025A0780126654A59
:1033B000103305287ED2DFE800F00313113E110020
:1033C000108820F0010010801D805F480580001FDC
:1033D0000580001F0580FFF7CDFFA670BDE8F087D0
:1033E000594941F244401C390880574945F6580074
:1033F00024390880091D47F25800088052492020CE
:10340000283908800020401CC0B27328FBD3FFF786
:10341000B1FF4C4984F85C502C3147F6906008802D
:103420004848143006801D80108840F0010010804C
:103430000220A070D2E700215FF0010004EB4102FE
:1034400004EB4003B2F85020B3F850309A4200D257
:103450000146401CC0B20628F0D33C48405C84F8CA
:103460003900FFF74DFF1D2000F0F3F900F076F86A
:10347000374E38484FF4807996F83B10012904D034
:1034800002291BD0042930D047E040218046FEF7B6
:103490004BFF870080214046FEF746FF47EA400782
:1034A00049464046FEF740FF074347F0010084F8D5
:1034B0003B0000E03DE0224809302CE040218046FE
:1034C000FEF732FF870080214046FEF72DFF47EAD6
:1034D000400749464046FEF727FF074347F00200F2
:1034E00084F83B001648133015E040218046FEF773
:1034F0001BFF870080214046FEF716FF47EA400782
:1035000049464046FEF710FF074347F0040084F8A1
:103510003B000B481D3002F08FFD94F82F0086F819
:1035200038001D2000F0ABF90420A0700A48057097
:1035300054E7108820F0010010801D80A5704DE731
:1035400034040020000800403C2C0140E4880008BE
:103550003401002000100140E70600202DE9F04171
:10356000344C14F82F0F344DE07240212846FEF7FA
:10357000DBFE860080212846FEF7D6FE46EA40069E
:10358000AF1539462846FEF7CFFE0643207BF1B241
:103590002F3C814215D084F83C0040212846FEF79C
:1035A000C3FE860080212846FEF7BEFE46EA40069E
:1035B00039462846FEF7B8FE064384F83B60FFF71D
:1035C00065F81E4D95F83B00012827D0022828D029
:1035D000042829D0174894F83B102730085C04F8D9
:1035E000300F14F80109FEF72BFF04F82F09A87A11
:1035F00000B10120607001F0D3F994F84E0094F806
:103600003B10884206D094F83800062802D2401CAD
:1036100084F8380084F84E10BDE8F0810548093080
:1036200004E00448133001E002481D30BDE8F041D9
:10363000FFF7F4BD340400200010014034010020E5
:103640002DE9F041524991F87200AA287ED191F8F3
:10365000730055287AD14F4C00200A5C2254401C3C
:10366000C0B27428F9D34C4E2069C6F80100A08A74
:10367000A6F80500D4F81600F060D4F81A003061FE
:10368000D4F81E001234706102F07CFC4349608A59
:10369000888102F091FC207D123CC007307802D076
:1036A00040F0040001E020F004003D4930704FF488
:1036B00080403C4D886114F8280F85F82000608B0D
:1036C0006880A08BA880E08BE880208C2881608CAB
:1036D000354F688194F8240087F8D20014F8011C53
:1036E000304686F83B100026C0F89460FFF724FEB1
:1036F0002E48A18E0183E18E4183218F818394F82E
:103700004210283C012908D0022901D0032909D000
:10371000297821F00C01083107E0297821F00C010B
:10372000091D02E0297841F00C01297094F86E20FF
:10373000012162B1012A01D0022A0BD087F846107C
:1037400094F864301A4A4BB1518108E014E087F8CC
:103750004660F5E7022287F84620F1E7568194F8A3
:10376000701001290AD094F86D1051B101290BD0C5
:103770004FF48051A0F87610BDE8F08144F21C713E
:10378000F8E74FF40051F5E741F25551F2E7000038
:1037900000FC0008540C0020340100205C000020D4
:1037A000EC0B0020AC040020900200201405002047
:1037B000000A00207CB50121082000F0ADFB4FF489
:1037C0008070ADF8040010248DF8074001208DF8BA
:1037D000060001A91548FEF729FD0121092000F086
:1037E0009BFB01211248FEF773FD0820ADF8000095
:1037F00004208DF803000F4E03258DF80250694612
:103800003046FEF713FD08213046FEF794FDADF873
:1038100000408DF803408DF8025069463046FEF7AF
:1038200005FD10213046FEF786FD7CBD00140140E9
:1038300000023000000C0140FEE7704700F01F025C
:10384000012191404009800000F1E020C0F8801182
:10385000704700F01F02012191404009800000F1F3
:10386000E020C0F88011704700F01F020121914054
:103870004009800000F1E020C0F80011704700F01E
:103880001F02012191404009800000F1E020C0F8B2
:103890000011704770B50F23C47801780122F4B18C
:1038A000144C2468457804F4E064C4F5E064240A08
:1038B000C4F10406E3408478B5401C402C4301F178
:1038C000E021230181F80034007800F01F018A40D4
:1038D0004009800000F1E020C0F8002170BD01F037
:1038E0001F0082404809800000F1E020C0F88021DC
:1038F00070BD00000CED00E0024908430249086079
:10390000704700000000FA050CED00E02DE9F05FC3
:1039100000261D20FFF792FF6C4CDFF8B4B1A4F134
:10392000B000A77E90F83810DFF8A8E1DFF8A8A172
:1039300000258F427ED0E776A176626A036B5A43F8
:103940004FEA12499BF80820120702D51EF8012001
:1039500000E00A4694F812C0BCF1010F09D004EB54
:103960004206B6F902C0C4F828C0B6F90460E6629F
:103970000CE043F6FF7CC4E90A5C90F83DC05FEAC6
:10398000CC7C01D012B102E0052A00D1012600EB67
:1039900047074FF0804CBF893F04B7FBF3F3E36167
:1039A000476BBCFBF7F7276294F813C0BCF1000F1C
:1039B00006D0BCF1010F05D03B4403EBD3735B1081
:1039C000636201E03B466762DFF810C14FF6FF77A4
:1039D00007EA8307ACF808709AF8007090F80A803C
:1039E00090F83DC0082F08F003070CF0030C05D039
:1039F00067450BD1B8F1000F05D008E0674505D049
:103A0000B8F1000F03D05B42636200E06562C6B1AB
:103A1000636A002B03D006DD228D05E00AE0304BFF
:103A200033F8122000E0A28DA4F86020227822F062
:103A3000200222709AF80020042A07D0082A05D014
:103A400012E0B4F8603003EB0902EDE780F8405073
:103A500065629BF80800000701D51EF80110204898
:103A600030F81100A4F860001E49606A09883E31F0
:103A70004843B4F8601001EB204006B21D20FFF768
:103A8000F3FE606A002807D021784FEA81600ADDE2
:103A9000002804DAA08D09E0B4F8600006E0E06ACE
:103AA000B04208DB0CE0002802DA208D208208E01A
:103AB000A06AB04204DD208241F02000207000E0C6
:103AC0002682257565752586BDE8F09FE4010020F6
:103AD0009002002018910008E7060020D809002075
:103AE0002A9100082404004043184FF48042934276
:103AF00010DD904202DD104600210BE0914202DD14
:103B00000020114606E08003B0FBF3F000B2C0F5E0
:103B1000804109B241EA0040704700002DE9F043BE
:103B2000002340F22D440E2544600362058143F6D4
:103B300032360827C6600782DFF8349043F6FF7CF0
:103B4000A0F81290A0F814C04FF070484FEA8C32E1
:103B5000C0E906824C600B620D81CE600F82A1F835
:103B60001290A1F814C0C1E90682BDE8F0830000FC
:103B700000C0FFFF00214162094981600E2181815F
:103B800008490161082181824FF44041C18243F616
:103B9000FF7101830907C161034901627047000099
:103BA000B7B90100331C010000C0FF0F064941F600
:103BB000A260088005480168054A01F4E0611143EC
:103BC0000160BFF34F8FFEE7442C01400CED00E095
:103BD0000400FA0538B501210D2000F09DF94FF4DD
:103BE000E060ADF8000018248DF8034003258DF83F
:103BF000025069460D48FEF719FB4FF46040ADF8DE
:103C000000008DF803400A4C8DF8025069462046AA
:103C1000FEF70CFBA014ADF8000048208DF803005F
:103C200069462046FEF702FB38BD0000000801404F
:103C3000000C0140F0B50121CE028DB0304600F0FD
:103C40006BF9594F384601F01DFB08A801F046FDFD
:103C50004FF45860ADF824000024ADF82040202037
:103C6000ADF82200ADF8264008A9384601F0E8FC7E
:103C70000021384601F03BFD4FF6FF71384601F058
:103C800040FD01220021384601F0CCFC01213846DC
:103C900001F0B4FA04A801F0CCFAADF8106070108D
:103CA000ADF81200ADF81440A220ADF81600700077
:103CB000ADF81800ADF81A40ADF81C4004A938461C
:103CC00001F0A6FA6025ADF80050ADF80440ADF85B
:103CD0000840ADF80C40ADF80240ADF80640ADF834
:103CE0000A40ADF80E406946384601F08BFB694644
:103CF000384601F0CDFB6946384601F013FCADF8BB
:103D000000500125ADF8045040F61450ADF80600FF
:103D1000ADF80840ADF80C40ADF80250ADF80A40DF
:103D2000ADF80E406946384601F040FC01213846A6
:103D300001F088FA0821384601F0A4FB31463846E4
:103D400001F0E6FB0821384601F02AFC31463846EE
:103D500001F05EFC7021384601F067FC18208DF8F8
:103D60002C008DF82D408DF82E408DF82F500BA88B
:103D7000FFF790FD0C480C30018841F08001018074
:103D800009481430018841F001010180001F0480BE
:103D90000121384601F060FA8DF82850012138469B
:103DA00001F064FA0DB0F0BD002C01407047000036
:103DB00070B50189C1EB411101EB4101CA0B428190
:103DC0000B49104603F0B6FC09480C38B0F90C203A
:103DD0000168B0F90E4001FB02F54368614303FB43
:103DE000145503FB0211AD138913C0E9055170BDD1
:103DF000E409002040F213414160082181608621DE
:103E0000C1604FF48041016149424161002101627A
:103E1000C16270470162704710B501884288891AF3
:103E200009B20183B1F5005F02DBA1F5804104E036
:103E300011F5005F02DC01F580410183B0F9182023
:103E400041685143C1618368846A5343C2681B124D
:103E5000624303EB2222036A1A44114402628A136A
:103E6000426241698A4203DB01698A4200DC1146F1
:103E70008A1AC0E90A21028E4FF40373594302EBF8
:103E8000A13202860B4A1278082A04D10A4AD36E5C
:103E900003EBA131D166B0F93010B1F5804F02DDEE
:103EA000A1F5804103E0002902DA01F58041018695
:103EB00010BD0000E7060020140A0020034A5168E4
:103EC00021F440410143516070470000001002405E
:103ED000044A0029516901D0014300E08143516146
:103EE0007047000000100240044A0029D16901D047
:103EF000014300E08143D16170470000001002409F
:103F0000044A0029116901D0014300E08143116195
:103F10007047000000100240044A0029916901D056
:103F2000014300E0814391617047000000100240AE
:103F3000044A0029D16801D0014300E08143D160E7
:103F4000704700000010024030B524494A6812F062
:103F50000C03234A03D0042B01D0082B26D0026087
:103F60004A680F231F4C03EA1212A35C0268DA406E
:103F700042604B68072505EA1323E35C22FA03F34A
:103F800083604B6805EAD323E35CDA40C2604B6888
:103F9000032403F4404104EA933303EB9161114B92
:103FA0001B1F595CB2FBF1F1016130BD4A680E4B39
:103FB0001A404B68140103F4803303D5C2F38342E3
:103FC000113202E0022404EB924213B14B689B03CE
:103FD00001D5064B00E0024B5A43C0E700100240F7
:103FE00000127A000400002000003C0800093D0097
:103FF0002DE9F041274CA61540212046FEF794F903
:10400000850080212046FEF78FF945EA40053146BC
:104010002046FEF789F90543EDB240212046FEF720
:1040200083F9870080212046FEF77EF947EA4007A2
:1040300031462046FEF778F90743F8B2A842DBD1B3
:1040400040212046FEF770F9870080212046FEF7C8
:104050006BF947EA400731462046FEF765F907430A
:10406000F8B2A842C8D140212046FEF75DF987008A
:1040700080212046FEF758F947EA4007314620469E
:10408000FEF752F90743F8B2A842B5D12846BDE879
:10409000F08100000010014010B50268416802FB89
:1040A00002F301FB01330D4CA34211D91B0E0C3B53
:1040B0000B4C9BB212B234F8133009B25A43594335
:1040C00042F38F3241F38F31C0E90221012102E036
:1040D000C0E902210021017410BD0000A4F0F50C1C
:1040E0006C8600082DE9F05FFE48FF4902880B88C6
:1040F0009A1A92B20F2A77D309880180FB480246A8
:104100008189D2884B0703D48B0701D4CB0702D017
:1041100042F4007201E022F40072C2808346080774
:1041200002D45846C90604D5BBF8061041F0010177
:1041300002E0C18821F00101ABF80610EB48FDF761
:1041400077FEEB484FF48049B0F93A10494502DA5E
:10415000491C418702E0E649A1F83A90E54E41F654
:10416000CC41E54CB06C884203DDA06820F0100023
:10417000A060E24AE24FE3481188002511B1491ED0
:10418000118008E0E18F41B1491EE187DE490A78DC
:1041900022F002020A70E5732DE0BBF806104B0412
:1041A00019D4BBF80C20D30615D4120713D40A0671
:1041B00011D48A060FD40A050DD44A0603D5D34A72
:1041C0001278120607D54A0705D4CA0503D40A0790
:1041D00001D4C90609D5CE49E573CE4A3D70CD83D9
:1041E000158081F82A5007E07BE03978012903D156
:1041F0000178062900D13D703A78DFF8FCA2C64963
:104200004FF00108AAF12C0A0A2A78D2DFE802F05E
:1042100077690569F9F86977E4FEE07B09281AD027
:10422000DFF8F8B202286CD0B4F8400010B39BF865
:10423000680040F63A22012822D0C4F8D85084F809
:10424000EA50CAF82050B4F9301001F21D509042E3
:1042500026D8102325E0A3484430FEF751F9FDF796
:1042600091FE716CCAF8281041F27C510920CAF8FD
:10427000181075E1AA48808A2086A4F8408015E0CD
:10428000A848C4F8D80084F8EA80B4F9301001F2E4
:104290001D53934201D8102300E02023102202E096
:1042A00020231022002000F0E5FA20869BF86830D9
:1042B0009D48012B736C40F2DC514FF4A37212D075
:1042C0008B4204DA9649B1F90A10914212DDB4F832
:1042D000401040F6C412491C89B2A4F84010914223
:1042E00008D2BDE8F09F8B42FBDA8D49B1F90A1084
:1042F0009142F6DC3D7084F8EA504583F1E7AFE087
:10430000FFE7706CCAF828008AF80780874FA4F886
:10431000405084F8EA50797F5646C9B1F87FE0B33F
:10432000208DB4F9301000B20A23052200F0A2FA61
:1043300020866F4840F6CC418068884201DDFD77D9
:104340007D77B4F93000484542DDA4F83090C8E7E5
:1043500000B2774901F0DCFBA4F8E400A26A8242D3
:1043600000DA1046B0829BF84D00B4F930100028F6
:104370005F4610B201D0362301E040F24713052218
:1043800000F078FA2086B4F91601B4F914118842C5
:104390000ADA97F84D1021B100E015E000F10200B3
:1043A0000CE000F1080009E00BDD317901F10101B9
:1043B000C9B231710229C4D33571401EA4F8160167
:1043C000BFE7A4F81611BCE740F266602086B8E7A4
:1043D000002886DA258684E75649D4F8DC0088422E
:1043E00002D2401CC4F8DC00E07B082803D1D4F8DA
:1043F000DC00884206D33D70C4F8DC5071E705E06C
:104400002AE025E0BDE8F05F02F0D6BBE07B09289A
:1044100001D0258604E1DAF81C005746401CCAF892
:104420001C00022809DD388D012301B2388B0522DA
:1044300000B200F01FFAFD61B8622A48398D44309D
:104440000180B6F844104180FEF772F8208648E7F4
:10445000BDE8F05F03F0CCBF0878092870D040E7D2
:10446000E27B921E082A6CD2DFE802F006A0DCEDA7
:1044700005F77C04EFE634E7FDF790FF307840065F
:1044800011D52D48807804280DD0706C82280ADA66
:10449000B07A96F83D1000F0030001F00301884265
:1044A00001D001F035FD3878062894D086F83F50C9
:1044B000B06C1B4940F31100886281031F48016200
:1044C000FDF760FD8AF80780B4F81401A4F816011E
:1044D000706CA4F88250B0F5437FA4F880907DDC26
:1044E000A1682FE010090020F0060020000A00203B
:1044F000140500203401002090020020F406002062
:10450000E7060020E8060020BE050020C8060020BF
:10451000A40800201A0000204C020020540C0020A7
:104520005C0000209AF9FFFF800900201C0C00208D
:1045300026880008C0D40100340400208008002030
:104540006EE08AE021F48061A16040F28A21884215
:1045500004DA3078400601D402F01AFAA0685AE072
:104560003870BEE6716CB1F5437F04DA0178062934
:1045700001D005706AE03C48017821F040010170EB
:10458000FDF700FDA4F81691FDF708FF374810F875
:10459000281F21F0010101703549C4F8DC500D627B
:1045A00034490D620821397045649AE69BF806008B
:1045B000C006D6D4706CB0F57A7F31DDFDF7EEFE23
:1045C0003078400613D52C48807804280FD0706CC2
:1045D00082280CDAB07A00F0030000E013E096F8CD
:1045E0003D1001F00301884201D001F091FC86F8F2
:1045F0003F50B6F84800208601B2494501DDA4F8D5
:104600003090FDF7BFFCA06840F48060A06096F891
:1046100038100529A5D140F01000A06002209FE7C6
:104620003D705EE6716CB1F5437F02DA01780629D0
:104630009FD1BBF8061021F02001ABF80610FDF762
:10464000ADFE04208CE70078062802D087F80080B1
:1046500047E609200870052082E707498D7005703C
:10466000064880F85250B5E6F6060020140A0020ED
:104670005C08002080080020340400205C0000203A
:1046800030B585B001210420FFF746FC4FF400400F
:10469000ADF8100048208DF8130004A91848FDF764
:1046A000C5FD01210846FFF71FFC40F68C20ADF840
:1046B000040003240020ADF80040ADF80200ADF87E
:1046C00006004FF080456946284600F0B9FF1C20DF
:1046D0008DF80C008DF80D408DF80E4001208DF8FE
:1046E0000F0003A8FFF7D6F801221146284600F074
:1046F00081FE0121284600F0AFFD05B030BD00006D
:1047000000080140704700002DE9F041304CE0788E
:1047100000285AD12078002857D0401E10F0FF0002
:10472000207052D14FF49670208272B6294F45F214
:10473000AA50A7F872000020FDF702FC264D1320B6
:104740002860FDF70FFCA8BB3420E8600220286138
:10475000224E6E61286940F040002861FDF702FC9E
:1047600040BB00211E4A08465FEA255312F800C0EC
:10477000BCF1FF0F00D00121401C80B29842F5D35C
:10478000C1B9C4E9067639260127A06910F8011BD2
:1047900010F8012BA061E06901EB022102886A6137
:1047A0002F6120F8021BE061FDF7DCFB10B9761EDB
:1047B000B6B2EAD20120FDF7C3FB62B601F0FCFB02
:1047C0000848816821F480418160BDE8F0810000E3
:1047D000E4060020540C00200020024000FC0008E9
:1047E00000FC0008900200201948016841F0100107
:1047F0000160016821F003010160016841F00201DC
:10480000016014484168416041684160416841F479
:1048100080614160416821F47C11416041680E4A29
:1048200011434160016841F08071016001688901B4
:10483000FCD5416821F003014160416841F002016B
:1048400041604168C1F381010229FAD1704700003B
:1048500000200240001002400000280830B5044C3F
:10486000039D6080A180E2802381658130BD0000CE
:10487000F40900200A44824201DA10B27047C91AD2
:104880008142FBDD08B27047F0B53E48DFF8F8E042
:104890003E4CC17F467A056800233D4A3D484FF0B3
:1048A000010C802925D301F01F015EF821100D4273
:1048B0000146096802D041F4805101E021F48051A1
:1048C0000160CF0411D48F040FD5977AFF0705D06C
:1048D0005381277827F00207277006E090F846708A
:1048E0009FB1012F14D080F846300F0B67F34D3184
:1048F0000160802E25D306F01F015EF821100D42C5
:10490000016809D041F0040108E080F846C0ECE7F6
:10491000022780F84670E8E721F0040101604D07A6
:104920000BD44D0509D5957AED0706D0538125782E
:1049300025F002052570C0F898308C0864F38A21B0
:104940000160917AC90718D1134991F864100129BF
:1049500013D11249496C32290DDC017849070AD577
:104960000189090507D4D0F8981047F23054A142C4
:1049700004D9A2F80AC0C0F89830F0BD491CC0F8AC
:104980009810F0BDC40500204C8D0008BE05002025
:10499000000A002090020020540C00203401002066
:1049A00010B5FCF7E5F90F48018821F002010180FC
:1049B0000C49183109880C4A928E1144094A343244
:1049C000118008490C390A8842F001020A80011D51
:1049D0000A884FF6ED531A400A80018841F012010F
:1049E000018010BD0C0400403404002006480188FA
:1049F000491C89B20180B1F57A7F04D34188491CF2
:104A00004180002101807047080700200F4810B541
:104A1000016841F00101016041680D4A11404160A7
:104A200001680C4A11400160016821F48021016095
:104A3000416821F4FE0141604FF41F018160FFF7DE
:104A4000D3FE05494FF00060086010BD0010024021
:104A50000000FFF8FFFFF6FE08ED00E02DE9F04151
:104A60002F4D28884FF00004000629D5FCF7FAFAEC
:104A70002C4A2D4807231778C8262C49012F22D00D
:104A80002B4FB7F806C0BCF1000F3ED0B0F80CC0F9
:104A90004CF0080CA0F80CC0B0F806C02CF4006C68
:104AA000A0F806C0886820F004008860FC801370BD
:104AB000CE8700204FF49661401C80B28842FBD321
:104AC0002C80BDE8F0811B4F97F800C0BCF1010FAE
:104AD0000FD0BCF1020F11D0B0F806C04CF4006C3E
:104AE000A0F806C0886840F004008860052038708F
:104AF000DDE7B0F80CC04CF0080C03E0B0F80CC0D7
:104B00004CF0100CA0F80CC0F0E70B4F3C70C788BD
:104B100047F40067C780886840F004008860C6E7F3
:104B2000102C0140E7060020000A0020900200201F
:104B300010090020E806002005070020704700004B
:104B40002DE9F0434FF08040018A21F001010182FC
:104B5000AC48007800287CD1AB4FF87B002878D196
:104B6000AA48406C322874DCA9488068DFF8A49217
:104B70004104A94DB9F804004FF0000403D4401CCF
:104B8000A9F8040028E1002874D02978012611B181
:104B9000012912D017E14946B0F5BE7FFAD92E702F
:104BA000CC718C71EC702C72287A0A18401CC0B23F
:104BB000147228720F28F7D305E1B9F8022049468C
:104BC000824201D9EE7100E0EC7192488A79083096
:104BD0000F2A15D2CB79082B0BD2C3F10708EB793A
:104BE00012F800C003FA08F363441354CA79521C44
:104BF000CA71CA79082A03D18A79521C8A71CC7188
:104C000099F80610C8460F2973D10D21FCF794F9C5
:104C1000A881010A6970C0B2A87088F8064098F8A7
:104C200016208A4265D198F81510814261D198F812
:104C30000BC07A49032302227948BCF1000F10D03F
:104C4000BCF1010F02D0BCF1020F14D080F86A2031
:104C500000E0CBE091F800C02CF00C0C0CF1080C3B
:104C60000FE080F86A6091F800C02CF00C0C0CF199
:104C7000040C06E0A9E080F86A3091F800C04CF01E
:104C80000C0C81F800C098F80C10B6EB111F04D181
:104C900080F86E4087F846400EE0B2EB111F04D159
:104CA00080F86E6087F8466006E0B3EB111F03D111
:104CB00080F86E2087F846200B0717D001F00F010F
:104CC000012901D0022915D080F86C602C7198F868
:104CD0000D102A7906FA02F30B406B71082A44D2B0
:104CE000DFE802F00B124319242F363D80F86C40A8
:104CF000ECE768E080F86C20E8E713B180F87040DA
:104D000033E080F8706030E013B180F850602CE040
:104D100080F8504029E023B180F8656087F803618E
:104D200023E080F8654087F803411EE023B187F84F
:104D3000F54080F84D4018E087F8F56080F84D6048
:104D400013E013B180F868600FE080F868400CE071
:104D500013B180F8666008E080F8664005E013B1A2
:104D600080F8676001E080F86740521CD2B22A7177
:104D7000082AAED398F80E102A4A8B0705D587F873
:104D8000F16080F86460568104E087F8F14080F8B3
:104D900064405481C90702D080F8294001E080F8BE
:104DA000296098F8111000F86D1FC2781E48012A7A
:104DB0001ED001B3012921D04FF48051A0F8761004
:104DC0001A493C200870A9F80240A9F80440B9F833
:104DD0000210491CA9F80210B9F80210B1F5FA7FC7
:104DE00004D940F2F511A9F802102C70BDE8F08347
:104DF00044F21C71E2E74FF40051DFE741F25551F4
:104E0000DCE70000E70600209002002034010020CB
:104E1000001001403C0C002080060020AC04002063
:104E2000540C0020000A002014050020E406002095
:104E30002DE9F05FFDF7B2FA8E4D2888A5F1040642
:104E4000C0070AD0308820F008003080288820F081
:104E50000900288001F09CFDD9E02888DFF818922D
:104E6000DFF81882864C80071AD5B9F8001041F097
:104E70000101A9F80010B8F8000080491431503041
:104E8000088028884FF6F95108402880308840F083
:104E900004003080FFF7ACF884F83C00BDE8F09FD8
:104EA0002888784F4007288871D520F00400288092
:104EB000FFF79EF894F83C108142EFD1308820F043
:104EC00004003080FDF742FC2078410605D594F8B7
:104ED0004C1094F83B209142E0D03978400621F004
:104EE0000201397004D5FEF739FB97F82F7004E002
:104EF00094F83C00FDF7A4FA0746DFF880B140F6CD
:104F00008C2A0BF1180B062F47D294F83800B842C0
:104F10003ED03846FDF718FA2078C00716D094F82E
:104F20003A0094F8391000F00302914206D0A17AB9
:104F300000F0010001F00101884215D1FDF76EFB80
:104F4000FBF762FFFDF796FC384689E0FDF766FB4C
:104F5000FBF75AFFFDF78EFC3846FDF77FFB207804
:104F600040F00100207099E7288820F00800288090
:104F7000206B810801EBD000504515D2B8F8001025
:104F80000844ABF80000308840F0080003E00DE072
:104F9000308820F00800308080E7B9F8001041F038
:104FA0000101A9F80010DFE75046E7E7000728886D
:104FB00031D520F008002880308820F008003080AB
:104FC000FFF716F884F83C00FDF7C0FB387820F0B6
:104FD000020038702078400604D5FEF7BFFA97F833
:104FE0002F5004E094F83C00FDF72AFA0546062D00
:104FF00008D294F83800A842B5D0FDF70FFBFBF7B4
:1050000003FF2AE02048C18841F04001C180BDE88B
:10501000F05FFDF70FBCC006288825D520F01000F2
:105020002880308820F01000308097F838000C2855
:1050300002D2401C87F83800387840F002003870FF
:10504000FEF78CFA97F82F50787884F8390094F8A6
:105050003800A84287D0FDF7E1FAFDF70BFC28469F
:10506000BDE8F05FFDF7FABA4EF2BE1108402880A5
:1050700014E7000010040040000400402404004035
:105080003401002034040020000A00202DE9F04FF4
:10509000514F85B0388820F0010038804E480026F6
:1050A000103006804D4CDFF838A14FF0010894F81D
:1050B0005C0042F63029C10774D072B64948816954
:1050C00041F400718161816941F4806181614FF433
:1050D0000040FEF7F3FE444D00212846FBF7F2FBAB
:1050E00000212846FBF7E4FBDFF800B10021584619
:1050F000FBF7DEFB00213E48FCF76EFA2846FBF783
:10510000FDFC5846FBF7FAFC4FF46020CDE902069F
:105110008DF8056000968DF810808DF80480694642
:105120002846FBF77DFD01231A460F212846FBF791
:10513000C8FD01212846FBF7BBFB00204946401C67
:1051400080B28842FBD328462E600121FBF7F8FD90
:1051500028688007FCD524484C30006894F85C101F
:1051600021F001012144A1F85000FBF7B5FB62B624
:10517000FEF700F947F69061AAF8001094F85C0079
:10518000401CC0B284F85C000C2822D212491431B1
:10519000A1F80080388840F00100388005B0BDE8F3
:1051A000F08FFFE7134920F00100085A12490880E8
:1051B000114945F65800083908800F4847F2580150
:1051C000001F01800C4920200C390880AAF80090AB
:1051D000D4E70320A070E1E7000800403404002079
:1051E0002C0800400010024000240140002801402B
:1051F0000800024008890008202C0140002901888D
:1052000002D041F0800101E021F08001018070476F
:1052100010B50A884B88CC881A438B8823431A43DD
:105220000B891A434B8989891A430A43A0F8442001
:1052300010BD0021018041808180C18001814181B8
:10524000818170470029818802D041F0010101E08D
:1052500021F00101818070470029018802D041F0CE
:10526000010101E021F0010101807047002930F8BF
:10527000441F02D041F4004101E0C1F30E0101805E
:10528000704700004B4910B5884202D10121C41477
:1052900086E0B0F1804F09D0474988420DD1012105
:1052A0000220FEF72DFE0021022064E001210846C5
:1052B000FEF726FE002101205DE04049884206D12C
:1052C00001210420FEF71CFE0021042053E03C498C
:1052D000884206D101210820FEF712FE0021082095
:1052E00049E03849884206D101211020FEF708FE26
:1052F000002110203FE03449884206D101212020BE
:10530000FEF7FEFD0021202035E03049884202D121
:105310000121441444E02E49884202D10121CC04E9
:105320003EE02C49884202D101210C0538E02A498F
:10533000884202D101214C0532E02849884206D139
:1053400001214020FEF7DCFD0021402013E024492C
:10535000884206D101218020FEF7D2FD0021802065
:1053600009E0204988420AD1841501212046FEF730
:10537000C7FD00212046BDE81040FEF7C1BD1A4917
:10538000884202D101210C040AE01849884202D166
:1053900001214C0404E0164988420AD101218C0401
:1053A0002046FEF7C5FD2046BDE810400021FEF76F
:1053B000BFBD10BD002C01400004004000080040AB
:1053C000000C004000100040001400400034014078
:1053D000004C0140005001400054014000180040C2
:1053E000001C0040002000400040014000440140FB
:1053F00000480140002A828901D00A4300E08A4324
:105400008281704730B5028C22F001020284028C46
:105410008388048B22F0020224F073050C882C434D
:105420000D8915434A882A43114DA8420BD0114DCE
:10543000A84208D0104DA84205D0104DA84202D075
:105440000F4DA8420DD122F008054A8923F440737C
:105450002A4322F004058A882A438D891D43CB897B
:105460002B4383800483C9888186028430BD000079
:10547000002C014000340140004001400044014044
:1054800000480140028B22F008020A430283704761
:1054900070B5028C22F010020284028C8488038B87
:1054A0000D8823F4E6464FF6FF7303EA05253543DE
:1054B0000E8922F0200203EA061616434A8803EA00
:1054C00002123243104EB04202D0104EB04215D1FB
:1054D00022F080064A8924F4406403EA021232432F
:1054E00022F040068A8803EA021232438E8903EAD8
:1054F00086062643CC8903EA8404344384800583EA
:10550000C9880187028470BD002C0140003401402D
:10551000028B4FF6FF7322F4006203EA012111436C
:105520000183704770B5028C22F480720284028C71
:105530008488838B0D8823F073031D4322F400734A
:105540000E894FF6FF7202EA06261E434B8802EAD6
:1055500003233343104EB04202D0104EB04215D157
:1055600023F400664B8924F4405402EA03233343B6
:1055700023F480668B8802EA032333438E8902EA90
:1055800006162643CC8902EA0414344384808583BA
:10559000C9888187038470BD002C0140003401401C
:1055A000828B22F008020A438283704770B5028C16
:1055B00022F480520284048C8288838B0D8823F429
:1055C000E6464FF6FF7303EA0525354324F40056FB
:1055D0000C8903EA043434434E8803EA0636264332
:1055E000094CA04202D0094CA04205D122F48044CB
:1055F0008A8903EA8212224382808583C988A0F8BF
:105600004010068470BD0000002C014000340140B1
:10561000828B4FF6FF7322F4006203EA01211143EB
:1056200081837047018582827047828822F07002F0
:10563000828082880A4382807047A0F840107047B9
:1056400030B502881B4B1C4C98420DD0A0420BD0A9
:10565000B0F1804F08D0194DA84205D0184DA8428E
:1056600002D0184DA84203D122F070054A882A437F
:10567000154DA84206D0154DA84203D022F440751E
:10568000CA882A4302808A8882850A8802859842CD
:105690000AD0A04208D00E4A904205D00D4A90424E
:1056A00002D00D4A904201D1097A018601218182FE
:1056B00030BD0000002C01400034014000040040D7
:1056C00000080040000C00400010004000140040A2
:1056D0000040014000440140004801404FF6FF7186
:1056E000818000210180C1804180017270470029C2
:1056F000018802D041F0020101E021F002010180A5
:1057000070470029018802D041F0040101E021F036
:105710000401018070470000214810B590F8201066
:10572000026801F01F001F4951F820001E49024283
:10573000086802D040F4803001E020F48030086036
:10574000C1031A484FF0000303D5194991F86510B9
:1057500021B3184902880C88A21A94B201220F2C96
:1057600008D30C8804808468042C03DD124C247850
:10577000022C05D0437F012B06D00988418010BD43
:105780004277C3770B88438043880988C91A89B256
:1057900040F21A639942F2D3C27710BD437710BD2D
:1057A000C40500204C8D0008900200201C0C002035
:1057B000540C0020F0060020E70600202DE9F04FF1
:1057C000DFF8B8B16A48DFF8AC91DFF8ACA190F827
:1057D0000EC0BBF91A70BBF91C60BBF91850BBF9BD
:1057E0006C10BCF1070F48D2DFE80CF08D041A30C2
:1057F000485E7600D9F800208284DAF80020C2845E
:10580000828CC38CA7EB820212B2A6EB83034A43BD
:105810001BB2594342F3CF2241F3CF23D11870E09A
:10582000D9F800204284DAF80020C284428CA5EB2B
:10583000820213B2C28C4B43A6EB820212B243F334
:10584000CF24514341F3CF23E11814E0D9F80020CD
:10585000C284DAF800204284C28C438CA6EB820218
:1058600012B2A5EB83031CB24A43614342F3CF2338
:1058700041F3CF24191949420AB244E0D9F8002073
:105880008284DAF800204284828C438CA7EB820267
:1058900012B2A5EB83034A431BB2594342F3CF2212
:1058A00041F3CF24111914E0D9F800204284DAF82A
:1058B00000208284428C838CA5EB820212B2A7EB7B
:1058C00083034A431BB242F3CF24594341F3CF220F
:1058D000A11849420BB216E0D9F80020C284DAF8C8
:1058E00000208284C28C838CA6EB820212B2A7EBCA
:1058F00083031CB24A4342F3CF23614341F3CF22D7
:10590000991849420CB2BBF91E50594605F21E5671
:10591000A64201DACE8306E0A5F21E55A54201DDBE
:10592000CD8300E0CC83B1F9204004F21E559542AE
:1059300001DA0D8406E0A4F21E54944201DD0C84C9
:1059400000E00A84B1F9222002F21E549C4202DADD
:10595000ABF8224008E0A2F21E529A4202DDABF8F8
:10596000222001E0ABF82230417B8173BDE8F08F4B
:10597000900200203C2401403C28014014050020F6
:105980002DE9F04704465748584D002602785648FE
:10599000022AB0F9301004D0082A7DD0092A07D095
:1059A00008E0C27B022A02D1B0F8402032B1E18780
:1059B00069812E8184F83C60BDE8F0874C49DFF8AE
:1059C0003481496A0F14E7808068410210D5B4F928
:1059D000020040F2DA21884269DD40F26A418842E1
:1059E0003FDCA0F2DA20FAF71AFD0022424B4BE02E
:1059F000C0F3C001C0F30020DFF8009181420CD158
:105A0000D8F8440040F2BA41884250DD40F66A11AD
:105A1000884226DCA0F2BA4032E039480078C0065D
:105A20000CD5D8F8440041F2243188423FDD41F2E0
:105A3000D471884215DC00F6DC401FE0314890F854
:105A40007010012903D090F86F0001282FD1B4F90C
:105A5000020041F6C811884229DD41F6786188428A
:105A60000ADD0823B4F93E101A460020FEF702FFB3
:105A7000E087002819DB1BE000F5C760A0F50050A7
:105A8000FAF7CDFC00224B46FAF735FC0E22FAF766
:105A9000A1FCFAF7FBFC00E01FE000B2C0F580407B
:105AA00078438013E087002F02DCE68700E0E78779
:105AB000E08F154FE880D8F844107964A7F84C00BF
:105AC00000F076FBB7F84E00688198F80A000028CD
:105AD000388F00D1404228816CE70C48B0F8700044
:105AE000688166E7E7060020900200205C00002045
:105AF00014050020340100200000794000C09240CD
:105B0000C8060020540C0020A4080020140A00201D
:105B10002DE9F041B1F9025000232B2415228542D2
:105B200003DAB1F90000BDE8F081B1F9AE50854269
:105B300002DDB1F9AC00F6E701EB8205B5F90250E0
:105B4000854201DD134600E01446E21852085D1C50
:105B5000AA42F1D101EB8206B6F90230834206DA9D
:105B600036F9025C36F9044C31F9221006E01D4684
:105B700031F92240B6F90630B6F90410401B091B72
:105B8000C6178911B60346EA90468703A1FB070CA6
:105B9000CA1702FB07C201FB06215A1BD317FAF7EB
:105BA000C3FA000A40EA0160001900B2B0F5804F64
:105BB000B9DB43F6FF70B6E770B5134C40F22445ED
:105BC0002946204600F03EF800281BD0204600F071
:105BD000C7F82946204600F01DF80C4C002120464D
:105BE000FBF7FAFC2046FBF775FDC0F1640008499D
:105BF000C0B20428087201D900F046F9BDE870402F
:105C0000FBF7AEBD70BD00000038014058000240F7
:105C1000500600200A0A01219140C94301807047C3
:105C20000029818902D041F4005101E021F40051A2
:105C300081817047002A828A01D00A4300E08A43AA
:105C40008282704730B501F01F0201240025C1F3A4
:105C5000421304FA02F2012B0FD0022B0FD0838AD9
:105C60004FEA11210088134204FA01F400EA04000B
:105C700001D000B10125284630BD8389F0E7038AB1
:105C8000EEE710B5C1F3421301F01F040121A1405A
:105C9000012B07D0022B07D01430002A026805D050
:105CA0000A4304E00C30F8E71030F6E78A4302605C
:105CB00010BD000030B50446008A85B00D464CF694
:105CC000FF710840E98801432182A1894EF6F31053
:105CD0000140A8882A8910436A890A431043A08199
:105CE000A08A4FF6FF410840A9890143A182684676
:105CF000FEF72AF91948844201D1039800E002987E
:105D0000A189090400EBC00101EB0010296801D54D
:105D1000490000E08900B0FBF1F06422B0FBF2F131
:105D200009010B096FF018056B4300EB8300A38991
:105D30001D044FF0320306D503EBC000B0FBF2F0B8
:105D400000F0070005E003EB0010B0FBF2F000F0FC
:105D50000F000843208105B030BD0000003801402D
:105D60008088C0F308007047F8B501210920FEF7CC
:105D7000D3F801218803FEF7CFF810258DF80350E2
:105D80002020ADF800001A4E03248DF80240694629
:105D90003046FCF74BFA16490C31086820F0200019
:105DA000086018208DF803004020ADF800008DF841
:105DB000024069463046FCF739FA48208DF8030066
:105DC0008020ADF8000069463046FCF72FFA8DF8C8
:105DD00003502801ADF800008DF8024069463046B6
:105DE000FCF724FA01210420FCF772FAF8BD000048
:105DF000000C014030B585B0FFF7B6FF00244FF42A
:105E0000E1300090ADF808400C201D4DADF8044085
:105E1000ADF80A00ADF80640ADF80C4069462846DA
:105E2000FFF748FF25208DF8100004208DF81100A1
:105E30008DF8124001208DF8130004A8FDF72AFD0B
:105E4000012240F224412846FFF71BFF012128468A
:105E5000FFF7E6FEFBF7AEFC012280212846FFF7A4
:105E6000E9FE012240212846FFF7E4FE012202213B
:105E70000448FBF743FCFBF79DFC05B030BD000078
:105E8000003801404400024070B51D4D00242878C0
:105E9000432834D16878462831D1A878502807D0D3
:105EA000512805D0812803D0892801D0212826D166
:105EB000144E7071E9787172A81C891CFBF774F894
:105EC000B072717A294409793182884217D106F17A
:105ED0000E00017841F0020101700B48016841F0A9
:105EE00020010160317A0948002204E02B5D03554E
:105EF0002A55641CE4B28C42F8D38078707170BD6E
:105F00007C070020500600200C0C0140860B00206E
:105F100070B51D20FDF79DFCFDF720FB1D20FDF752
:105F2000AEFC154890F82F10144D0623144C85F83C
:105F3000381090F83B1095F83B201143012A04D00B
:105F4000022A07D0042A0AD010E0827A8A420DD0B1
:105F5000007B09E0027D8A4208D0807D04E0827FD8
:105F60008A4203D090F82000884200D1237000209C
:105F700085F8400070BD000034040020340100208A
:105F8000E70600200B4800214180A0F1B0018A897A
:105F90008280CB891A44C2800B8A1A4402814B8AC0
:105FA0001A444281898A1144818143F6FF71C1817B
:105FB00070470000E4010020084940F61C72B1F966
:105FC0000C00904202DA00F59F7005E041F2E30216
:105FD000904201DDA0F59F70C88170475C000020F1
:105FE00038B51348C16941F00401C1611E208DF824
:105FF000000002208DF801008DF8020001248DF8C8
:1060000003406846FDF746FC0A4984200880094998
:1060100047F690602C3108800020091F0880054950
:1060200014310C80091F0880081F048038BD00004F
:10603000001002400008004030B420491E4A457854
:106040008B7A114692F83B4091F83910AC4218D146
:106050004BB10379994202D04379994201D14079F9
:106060001AE0807909E08379994202D0C479A1428B
:1060700002D182F82F3011E0407982F82F0030BC35
:106080007047C578AC42FAD16BB1C379994202D05E
:10609000037A994205D1007A82F82F0030BCFEF7CE
:1060A0007FBC407AE9E7437A9942E2D00479A14281
:1060B000DFD0007AE1E70000340400203401002042
:1060C000FEE700002DE9F0470446007F012868D173
:1060D0003548E1880288511A89B2072916D3008809
:1060E000E080B4F9000044F2DD414843401346F635
:1060F000D96148438013A060401000B2A0814FF0E6
:106100008051B1FBF0F0FAF785F92061B4F90C6029
:1061100096B1B4F902104DF6B05048430014A08275
:10612000B4F904704DF6B05207FB02F24FEA224573
:10613000E58204D4024603E00020E08330E04242DE
:1061400012B22283002D01DB2B4600E06B421BB212
:10615000DFF85890638398464FF4804AB24208DAD9
:10616000FAF74FF92169FAF722F8FAF776F980136E
:1061700004E0002901DA484600E05046E083B045DB
:1061800009DA2846FAF73DF92169FAF710F8FAF723
:1061900064F9801304E0002F01DA484600E050461D
:1061A0002084BDE8F0870000F006002000C0FFFF5B
:1061B00010B52348244C01782248022905D1C17B1F
:1061C000022902D1B0F8401029B1008EA4F84E0087
:1061D0000020208710BD90F846101B480229B0F817
:1061E000440000B201D0194923E019490978C1F3EC
:1061F000810101291CD002291ED014493039FBF736
:106200006FFE00BF1049A4F8400080B2483101F091
:1062100091FAB4F94C00B4F94A2041425143891330
:1062200024F8381FB4F9101048438013E08210BDE1
:106230000849FBF725FEE5E706496C31F9E7000060
:10624000E706002090020020A40800209C87000898
:10625000AC040020948600080348002180F82A102E
:10626000C183018770470000A408002010B5040016
:106270000B462D4AC3F1000028D56442002B12DAE8
:10628000A04207DA214600F027FA32F81000C0F5E4
:10629000404041E00146204600F01EFA32F810006E
:1062A00000F5004038E0A34208DA2146184600F025
:1062B00013FA32F8100000F540402DE0204600F0BF
:1062C0000BFA32F81000C0F5803025E0002B12DA0E
:1062D000A04207DA214600F0FFF932F8100000F57D
:1062E000804019E00146204600F0F6F932F810002F
:1062F000C0F5004010E0A34208DA2146184600F03D
:10630000EBF932F81000C0F5804005E053B12046AB
:1063100000F0E2F932F81000B0F5004F01DDA0F511
:10632000803010BD002010BD148900084043801348
:10633000494300EBA13000220302002B14DDB3F52A
:10634000001F01DC802001E04FF4005093FBF0F1CE
:10635000014401EBD1714910814206D0521CD2B2E6
:106360000846062AF2D300E00021C80000B27047B8
:1063700002E008C8121F08C1002AFAD1704770470E
:10638000002001E001C1121F002AFBD1704700006C
:106390002DE9F047A44CA54821880288511A89B2FA
:1063A0000F297DD30088A4F13C052080288F08B1F7
:1063B000401E28872B789E4AC3F3810001281DD0F8
:1063C000022820D0D18B98489A4FDFF86C92407EFB
:1063D0000026B1F5926F1DD8142819D37820607665
:1063E000F88840F01000F88040F26660A88123F041
:1063F00001002870D67389F8006015E0D08B00EB9F
:106400004000C00302E0D08B8C494843010CDAE71E
:10641000401C04E0B1F5DB6F06D310B1401E60767E
:1064200002E043F001002870B5F90200B5F914301C
:106430004143C3EBC303C1F38F31C3F3D10303EB78
:10644000510109B2A9829046D28B4FF0805350433C
:10645000B5F91620C0F38F30C2EBC202C2F3D102ED
:1064600002EB500000B2E882AA6A42431213EA62C9
:1064700093FBF2F22A63724A1080A2680A44A26077
:10648000E1680144E160207C401CC0B22074072810
:1064900006D942F3CF002883C9106983E66000E083
:1064A000BFE0A66041F6C8012674884204DD298B4E
:1064B000644AB2FBF1F1E981C117890341EA9041D5
:1064C000800342F69B420023F9F72EFEA88456482B
:1064D0002A78A0F13C005C49B0F90600930700FB64
:1064E00001F14FEA2141C2F3810215D5012A07D0FB
:1064F000022A0BD04FF2685141430914A18011E0E8
:1065000049F68C4250430014A0801FE04CF618312D
:1065100041430914A18025E0012A0DD0022A17D099
:10652000A0806984494948430014E083FBF7C8FA16
:1065300047480088C0B143E04AF65C324243121437
:10654000A2804BF62C22504300146884E183EDE7CF
:106550004DF2AC5141430914A1804EF27C414143BC
:10656000091469843B49DEE795F8200000BB88F8F0
:106570000F6089F80060B5F91A00A0F50C519F3939
:10658000B1F56E7F18D8617FF42912D93249E880BD
:106590002E4AA1F8460050430014A880A1F84400F8
:1065A000FF2085F8200081F828002C493C20087045
:1065B00006E0491C617703E0607F08B1401E607708
:1065C000B5F91A10B4F91E0081420EDDA07E7D28B7
:1065D00009D9F88840F00800F8802148017821F0B6
:1065E000020101700EE0401C06E0A0F23D10814265
:1065F00008DAA07E10B1401EA07603E0F88820F0F3
:106600000800F880B5F91810606908446061217EBF
:10661000491CC9B221761F2903D94011A88366619C
:106620002676BDE8F0870000E8040020F006002090
:1066300090020020000A0020E7060020303301000D
:10664000B409002074E8260BCC0E01004885010037
:10665000F2060020D0450100540C0020E406002082
:10666000BE050020024941F68B3088627047000069
:10667000AC04002070B5164C06252078062825D2DB
:10668000DFE800F003080E141A211248FAF7CAFCDA
:10669000012016E00F48801DFAF7C4FC022010E02C
:1066A0000C480C30FAF7BEFC03200AE0094812300F
:1066B000FAF7B8FC042004E006481830FAF7B2FCF8
:1066C0000520207070BDFAF7CDFC2570257070BDD7
:1066D000E806002008880008090A05D0B0FBF1F0A0
:1066E000FF2800D9FF20704700207047D0E9002123
:1066F000C368521A5A4301EBA2318160416070476E
:10670000B0F90020B0F90210B0F90630521A5A431D
:1067100001EBA2318180418070470000F0B54B4B06
:1067200018884B490A89801A85B24A484A4A0F2D6F
:10673000047801F148001DD31D880D81117A0F07DF
:106740000146B1F9021001F102052EB2A1F10205D4
:106750002DB20AD5022C01D0404909E0404FB7F9CB
:106760000070B9422CDC2FDB2CE0022C22D03D49FA
:1067700009884180818E1D88691A89B29C294FD36E
:1067800019888186936A0021B3F5804F3ADB364B36
:106790009B6CB3F5405F35DD344B40F26665B3F971
:1067A0001030AB421EDD43F69915AB420EDB40F2D2
:1067B000333315E02E4FB7F90070B94204DB01DD29
:1067C0004580D7E74780D5E74680D3E740F23335A9
:1067D000A3F2666303FB05F343F2333593FBF5F352
:1067E000038700E00187234BB2F806511B78C3F3FF
:1067F00081031DB1028F02F21E5219E092F8462069
:10680000022A0ED00187022C00D00187B0F9501067
:10681000B0F9382001F1140393420BDAA0F850309C
:10682000F0BD012B01D0022BE4D1028F02F23332F2
:106830000287E8E702F11403994203DD1439A0F856
:106840005010F0BDA0F85020F0BD0000F006002070
:1068500014000020E706002090020020AA04002077
:10686000A8040020A6040020340100201405002004
:10687000A4040020AC0400202DE9FC4101210220E9
:10688000FDF732FB01211920FDF746FB01213C48B1
:10689000FBF71EFD4027ADF8007003248DF8024081
:1068A0000420384D8DF8030069462846FBF7BEFCEE
:1068B000E001ADF800008DF802401C208DF80300C7
:1068C00069462846FBF7B2FC4FF4E0712846FBF717
:1068D00034FDA815ADF800008DF8024010208DF8A9
:1068E000030069462848FBF7A1FC4FF4A060FDF7C0
:1068F00003F81D208DF8040001268DF805600025A1
:106900008DF806508DF8076001A8FCF7C3FF1F49FA
:106910008C2008801D494FF6FA702C3108806E20BB
:10692000091F08801948143006801848083007806D
:10693000164920310D80154AD020121D1080134AAF
:1069400045F2F300183210800A1F45F25000108003
:106950000E4A4FF6FF7038321080121D1080121D43
:10696000108041F21B10088000F012F8FBF762FF64
:10697000064810300580001F0480BDE8FC8100003F
:10698000000C1A0000100140000C014000040040FF
:1069900070B51D20FCF752FF2A4D40212846FBF719
:1069A000C3FC840080212846FBF7BEFC44EA400477
:1069B000A9152846FBF7B8FC0443E0B2224C84F842
:1069C0003C00FBF73DFD0546052805D91F48C18859
:1069D00041F04001C18001E084F838501C48007A41
:1069E000000703D594F838001A490D5C4FF6FA7089
:1069F0002063E062A06260622062E061A0611648EC
:106A0000606300206064A06484F83F0084F8400064
:106A1000FBF7C4FCA07AFF2811D0022084F83D00C7
:106A20000E48008820662846FCF766F9207820F09A
:106A300001002070BDE870401D20FCF715BF01204B
:106A4000ECE700000010014034010020000A0020A3
:106A50009002002018910008DCFF0500240400408B
:106A60002DE9F0434E484F4902880B889A1A92B29A
:106A70000F2A69D3098801804B49098B027D00EBFD
:106A800042029180017D491CC9B2017508295BD37E
:106A9000002404752246017D00EB4103491CB3F933
:106AA0000430C9B202EB630212B201750829F2D3B5
:106AB0003E4904753E4B4A8044800E789D895FEACA
:106AC000C67C40F638694FF0030714D0A2F22B5C65
:106AD00042F6E858C44520D3A1F1020C26F0020486
:106AE000ACF8002047750C7040F22B54A24211DA2A
:106AF00045F004021EE046F001060E704A4507DD2F
:106B000045F001029A8126F002020A70477519E0E9
:106B1000447517E045F002020CE04A450CDA87752F
:106B2000427D12B1521E42750CE046F002020A701C
:106B300025F007029A8105E0B30703D5837D2BB1C9
:106B40005B1E837540888880BDE8F08342F6AA23E7
:106B50009A4222DAB1F904302BB941F2CD05AA42AA
:106B600001DA4480EEE7134C920302EB843241F6E3
:106B70007244B2FBF4F214B240F233350246448060
:106B8000AC4200DA5580B2F90240E41A04F5A3746D
:106B9000B4F5237FD6D84380D4E74FF48043FAE797
:106BA000880A0020F006002090020020BE05002088
:106BB000000A0020C8F1FFFF2DE9F0416C4CDFF81E
:106BC000B4E14FF0000594F82810C80706D094F9F6
:106BD0002C104B42002956DD0E4655E0664884F8DD
:106BE0002B50E586654A90F8380084F83400158605
:106BF000CEF80450CEF80850614E40F26663CEF8ED
:106C00000C50A4F8703036F810005E4E7688304490
:106C10004FF6FF7606EA800024F8240B4FF08060E0
:106C20002060A320208460845810A084E38440F670
:106C300099102085580060854FF48050A08541F25E
:106C40003330E08541F26660208641F69910608617
:106C500041F6CC40A0864FF40050E08642F233303B
:106C6000208742F26660608742F69910A08742F65C
:106C7000CC40E08782F89D5041F00100207184F8FB
:106C80004450BDE8F0811E4694F92B004242002892
:106C900001DD074600E01746F61B012E0BD0002849
:106CA00000DB02465FFA82F684F82C0094F8430079
:106CB000012805D041E0002900DA1946CEB2F3E7F9
:106CC00094F92D305942002B01DB184600E00846AC
:106CD00094F92E20C7B25042002A01DB944600E00E
:106CE0008446BC4508DD002A00DA0246D7B2002BF4
:106CF00000DA0B46D8B207E0002B00DA0B46DFB211
:106D0000002A00DB1046C0B204EB4000B0F944108A
:106D100004EB470030F9442F11444910018084F8F6
:106D2000435084F8325084F8315084F8305084F85D
:106D30002F5084F82E5084F82D5004EB46007546F1
:106D4000B0F94400E086BEF80410C82309B26422FA
:106D5000FDF790FD6860E968401AA9680844A860DA
:106D6000B5F900104843C013E860A4F8700088E744
:106D7000140A0020AC0500203401002090020020FD
:106D80002A9100085C0000202DE9F0415F4C94F846
:106D90002800C00779D05E4894F83410002690F897
:106DA00038005C4D814271D05B4AA4F866605B4F4D
:106DB000535C2246834292F92B2002D07B5C8342B3
:106DC0000FD1521C52B284F82B20795C814202D13F
:106DD000521C84F82B2094F92B100F291BDD0F2156
:106DE00017E04F4B5F5C4F4B874202D05F5C87429E
:106DF00011D1521E52B284F82B20595C814202D12B
:106E0000521E84F82B2094F92B206FF00E018A4239
:106E100001DA84F82B103D4994F833302D3194F881
:106E20002B205A5494F83310491CC9B284F83310FB
:106E3000062901D384F8336094F92D2094F92F109A
:106E40008A4211D194F9312091420DD194F92E202A
:106E500094F930108A4207D194F93220914203D13B
:106E6000012184F8431001E084F84360284984F844
:106E7000340094F92B300978012B0DDD254A4F079A
:106E8000926804D542F0080203E03CE015E022F0ED
:106E90000802AA6084F82900B3F1FF3F0ADA490723
:106EA000A96802D521F0080101E041F00801A960BC
:106EB00084F82900FBF772FA11E094F843000128E6
:106EC0000DD1B4F8660043F60951401C80B2A4F815
:106ED0006600884203D9A4F8666084F84360E87BC2
:106EE000082810D0B5F93010512341220020FDF7B9
:106EF000C1FC2886002806D10B48067014F8280F1C
:106F000020F001002070BDE8F0810000140A00208C
:106F100034010020900200200C910008129100081A
:106F20001E91000824910008E706002030B5204992
:106F3000204AB1F86A301088C01A80B20F2836D3C0
:106F40001088A1F86A001C4D00204FF000432A5C15
:106F5000940903D00124B4EB921F24D1D20622D08D
:106F6000164A52F820201268134C123434F810409C
:106F7000224201EB000494F9722008D00A2A04DBB3
:106F80000A6823FA00F4224308E0521C09E012F1D7
:106F90000A0F05DC0A6823FA00F4A2430A6002E043
:106FA000521E84F87220401CC0B21128CFD330BDCD
:106FB000C4050020F0060020188D0008188E000877
:106FC0002DE9F00779497A480A8903889A1A92B21A
:106FD000082A74D300880881A1F12C0042890AB1E3
:106FE000521E4281734A92F82820802A67D302F009
:106FF0003F020A70C2890AB1521EC281B1F906204D
:10700000902A0CDB8A46FF2A09D08146C0890028D5
:1070100055D1694800230078092805D005E0BDE86E
:10702000F007624800F096B90823644A92F8EA50E3
:107030000DB143F004036248817AC90701D043F0DF
:107040000203D2F808C05FEA0C5101D543F00103F6
:10705000176800215B4EFC0302D596F8654004B129
:107060008021C4885FEA446801D541F040015FEAAD
:10707000845801D541F020015FEAC47801D041F085
:107080001001007A400701D541F008014E48007810
:10709000C00701D041F00401A00601D541F0010173
:1070A0000020012D00D1082096F8705085B992F883
:1070B0004620022A04D0012A05D03AB108E072E045
:1070C00040F0030004E040F0020001E040F0010065
:1070D0007A0701D440F02000CCF3C0020025CCF3A5
:1070E000002C624502D13A0700D4042596F86F209F
:1070F000012A01D145F00105344A0027BC46127827
:107100003E46C2F38102012A04D0022A04D0032A97
:1071100004D004E0022602E0042600E010262C4AF7
:1071200064060ED5214C1C342478240609D5147825
:10713000640606D4274A40F6CC44926D6243140C90
:1071400005E0B2F8AE2040F699146243940B4FF07C
:1071500008088AF80A804FF061088AF80B808AF8DC
:107160000C308AF80D108AF80E008AF80F508AF851
:107170001070270A4B4083F06901414069408AF84A
:10718000117079408AF81240614052468AF813C063
:1071900071408AF8146051754FF4C871A9F80E1047
:1071A000FF20AAF80600BDE8F0077047AC060020F3
:1071B000F0060020C4050020E70600209002002011
:1071C000000A0020540C0020F8080020AC04002025
:1071D00034010020E00700204E48816941F0FC01A5
:1071E00081614FF4A060FCF787FBFBF7B1FBFCF774
:1071F000F1FCF9F7DBFCFCF7DDFAFDF741FAFFF7EC
:107200003BFBFCF71DFAFFF7C3FBFBF713FB424DFB
:107210004FF48040A5F81601FEF7ECFD00214FF475
:10722000FA5340F2EE220020401C80B29842FBD379
:10723000491C89B29142F6D33848002680F8726022
:10724000F9F74AFBF9F7E4FFFCF7F4FCF9F7B8FEAD
:10725000FEF7C6FE102232493248F8F796FF324C4C
:10726000334FE08820F04000E0803048017821F082
:1072700020010170FA20F8814FF49670E887FFF73B
:10728000F1F92C492C48FCF749FC2C48FCF772FC1E
:107290002B48416A88472B48416B8847FEF7DCFF43
:1072A0002948FAF708FC29494220C8802849C860C3
:1072B0003E71E088E0812089208260896082FAF74F
:1072C0002DFFFAF78FFEFFF763F8FFF7C9FB00F019
:1072D000F9F9FFF72BFE00F04FFFFEF71DFAFAF762
:1072E000BFFCFBF727FDFFF719FAFCF7FBFEFBF7E6
:1072F00049F9FBF77BF900F07BF8FFF761FE1248D4
:10730000FAF7A2FA00F070FAFDF7FEF9FAF70AFCB4
:10731000CFE700000010024090020020140500207A
:10732000540C002004060020000A00203401002034
:10733000E4060020800800205C080020F003002004
:1073400030000020C8000020800900200C07002029
:1073500020040020F0B523490278B0F9064000234C
:107360001F4E31F81210FF2C18D0B0F904701E4DCA
:10737000BC4231DA00EBE40704F00704BF7AA7400F
:107380008478FFB23CB190F801C0ACF1010C6445C7
:107390001FDA3C061DD455F822200DE056F82220B5
:1073A000116012498A79521CD2B28A71022A02D320
:1073B0008370C3808B71F0BD11608178491CC9B2A4
:1073C000817042789142F6D38370C188491CC18094
:1073D000F0BD56F82220EFE755F822201160F4E7BF
:1073E000F88E00082A8D0008A08E00088006002074
:1073F000F0B561486149B0F86C200B889A1A92B2D6
:107400009C2A7BD30988A0F86C105D495D4F91F8E8
:107410002A1001F0070297F84610022A00D1491EEF
:10742000594C80F83E104FF00203E2884FF0000103
:10743000550401D5012236E0A489E50601D50622CE
:1074400031E0250701D508222DE0550603D44F4D24
:107450002D78AD0601D5042225E0150501D50722BA
:1074600021E0150601D50A221DE0950601D50C2262
:1074700019E0150701D50B2215E0550701D4D505F4
:1074800001D510220FE0D50601D505220BE06507D6
:1074900003D4A50701D4E40702D080F86E3007E0DA
:1074A000920403D5032280F86E2001E080F86E106C
:1074B000374A384C92F820E0324A251FD2F808C0EB
:1074C0002D4AB2F87060721C92B2BEF1000F0DD05E
:1074D0002CF4000CC7F808C090F86E70B7B11E2FDE
:1074E0001AD090F86F200AB325E007E04CF40006AC
:1074F000BE60A0F870200A2A01D22360F0BD142AD1
:1075000001D22B60F0BDA0F87010F0BD2B60A0F888
:10751000701080F86F10F0BD642E04D2A0F87020B7
:10752000322AEED3E9E7A0F87010EAE77F1C80F872
:107530006F70A0F8701090F86F20012A10D0002A08
:10754000E9D0B0F87060761CB6B2A0F870601E2E5C
:10755000D7D323603C2EDED9521E80F86F20D2E7AD
:10756000B0F87020521C92B2A0F870202360C82A94
:10757000D1D980F86F10C6E7C4050020F0060020BE
:10758000540C002090020020000A0020340100204A
:10759000AC040020141C0140F0B54248B0F848107B
:1075A000491C89B2A0F8481002297AD33E49002428
:1075B000A0F848400A783D4B042A57D04FF4804148
:1075C000082A0BD0A0F10C02B2F900208A4200DA9E
:1075D0001146B3F980208A4200DA1146344A926992
:1075E0008A4200DA11B2418282881D8AC2EB85028A
:1075F000304D12B22D78C5F381062A4D42F2316624
:107600007243B5F9765092126A431213C2608668CB
:107610001546C6EBC60642F3D102F60202EBA632CD
:107620008260C66C1644C664B0F850707F1CBFB24E
:10763000A0F85070B7F5806F04D3B6120682A0F898
:107640005040C464891A1C4EC26A724340F25556B7
:107650004E4302EB4602466A32444262B3F930308E
:10766000B2EB034F06DD1A04426206E01349B1F99A
:107670000410B3E7002A00DA4462C162104990F8AE
:107680003D2091F838108A420BD080F83D10B0F8B8
:107690004210A0F84410B0F84010A0F84210A0F832
:1076A0004050F0BD14050020E706002090020020A5
:1076B000EC0B0020AC040020C3F5FFFF080C0020F9
:1076C0003401002017481849B0F85A200B889A1A3C
:1076D00092B20F2A25D30988A0F85A10134948F20C
:1076E000543391F84D10CA0701464FF48042B1F966
:1076F000001059430914A0F86C100D490B78A0F143
:107700000C01022B06D1B1F90030934202DA1B1DA5
:107710000B8000E00A800021A0F8601020F85C1FB8
:107720004280704714050020F0060020540C002011
:10773000E70600204FF6FF7202EA800210F4404391
:1077400015480ED0B3F5804F14D0B3F5004F4FEA73
:10775000122216D0C2F5807330F813305B424B8092
:1077600005E0120A30F812304B80C2F5807230F812
:1077700012000FE0120AC2F5807330F813304B800C
:1077800005E030F81230C2F580725B424B8030F871
:107790001200404208807047148B0008104A518A3A
:1077A000908AD28A16384639A2F1110200D5494290
:1077B000002A00DA52421144002800DA404208440C
:1077C000084943F6284300B2B1F936205A439213D0
:1077D00040F2D733584302EBA030C8867047000010
:1077E0009002002014050020F0B5904990480A89C5
:1077F00003889A1A92B23E2A1ED30088088101F1AA
:1078000038004FF4FA63428A9A4202D2521C4282F2
:1078100000E04382874A92F82220802A0CD302F0AB
:107820003F020A70B1F90620402A06DBFF2A04D085
:10783000C2883AB1521EC280F0BDBDE8F0407B481C
:10784000FFF788BD428A9A42F6D307784FF0010EBF
:107850003A074FF0FF055BD5847A40F2DC526307AC
:1078600008D444F004038372C28081F80BE081F8ED
:107870000AE04CE04378072B05D0032B03D0052BFF
:1078800001D0062B07D1660605D444F0400383726D
:10789000C280052239E0654A5FEA437C02F1380282
:1078A0004FF42076127A0DD55FEAC26C0AD45FEAF3
:1078B000446C07D442F0100202723A0628D4C68003
:1078C000192222E0DF0709D0970707D4670605D4FD
:1078D00042F002020272C680042216E09F0709D518
:1078E000170707D4670605D442F008020272C68063
:1078F00003220AE01B070BD5530709D4630607D4FC
:1079000042F004020272C6800B22CA728A72CD80D3
:10791000494AB2F92230B2F91A7003F23D1400223A
:10792000A74200DB0276414E444C06F13806A479AA
:10793000B6895FEAC46C06F101064FF4C874B6B2AA
:1079400013D58681B6F57A7F05D9017A21F08001B9
:1079500001728281F0BD037A1E06FBD4828143F05E
:1079600080020272C480112035E09F4216DA037E45
:10797000052B13D28681B6F5487F04D98281027A1D
:1079800022F040020272027A5606E3D45B1C0376B0
:1079900042F040020272C48002201CE0284B1C8985
:1079A000C4F3C006C4F3002740F2EE24BE4216D151
:1079B0001E78360713D4427E012ACBD1428BB2F512
:1079C000167F02D2521C4283F0BD827A42F002023C
:1079D0008272C4800F20C8728872CD80F0BD93F887
:1079E0000D714FF40046012F18D1164F41F6583C47
:1079F0007F6C674512DD83F80CE1134B1E60C38A70
:107A0000A34202D25B1CC382F0BD4FF4FA73C38061
:107A10001C23CB728B72CD80C282F0BDC2820A4819
:107A200083F80C21001F0660F0BD000090060020C6
:107A3000F0060020C4050020AC040020000A00204D
:107A40009002002034010020140801402DE9F05F6D
:107A5000DFF8FCB3FF489BF81830011D0A1DFE4CEF
:107A6000012B41D0B4F85A300380B4F85C00088090
:107A7000B4F85E001080FDF7A1FEF84FF84D49F212
:107A8000CD31B7F91E20EA82B7F92000DFF8D483A0
:107A900002EB4000484300142883B5F91E60B5F995
:107AA0001C3000FB06F102FB0311584302FB1600D9
:107AB000891369828013EC4EA882D8F844003060A4
:107AC000316930468847E949308948800846FDF7E2
:107AD00057FFE74E4FF0010A307808280DD0E98DA6
:107AE000298204283BD01BE0B4F860300380B4F84E
:107AF00062000880B4F86400BCE7DE4890F92B10FF
:107B0000491C022929D890F8681019B1B5F84E001F
:107B1000288205E0E98D2982A5F84E1080F868A03A
:107B2000B5F91410B5F90A00D34AF9F7ABFCA8620D
:107B3000B4F91611884204DDCF48A962027A914057
:107B40000162307804280DD0CB4AB5F91210B5F98E
:107B50000800243AF9F796FC08E0E88DD8E7786A3F
:107B60000014A86298F80A00A8B1C448C44F68621B
:107B70003860A86A78603846FCF71AF9BE4E387C3F
:107B8000383E01280AD0686A3060BE480178C907CB
:107B900008D0406907E04FF4AF70E7E778693060DC
:107BA000B86900E0A86A7060B3483838FCF774FA26
:107BB000AB4DAB4935F8100F3C39FFF7BBFDDFF893
:107BC000A092DFF8C482A9F14809D9F80C10C9F8CD
:107BD0006410B5F90C20B068B5F90E1000FB02F77F
:107BE000F368484303FB117646F38F3703FB02002B
:107BF00040F38F362F866E86A8F802704546A8F8A7
:107C000004604046FEF75EFA287F09F1100501285E
:107C100032D0704241104DF6B3504743381469805A
:107C200028800B18A9F80060A9F80230081AA9F8F2
:107C3000040000BF4FF0000884F80C80B9F9003050
:107C40004946002B01DD84F80CA0B1F902000028A0
:107C500002DD227B921C2273B9F90420002A02DD86
:107C6000217B091D2173217B072921D2DFE801F047
:107C7000201C3519311E3300B8F9203059424A1002
:107C80006A80B8F91E004DF6B351484301142980AB
:107C9000A9F800305318A9F80230511AA9F80410B5
:107CA000C8E784F80DA003E0022100E0032161731E
:107CB000DFF8AC91754E764F99F800100129617B81
:107CC0000DD007297CD2DFE801F0ECE9E8E7E6E532
:107CD000C2000421EBE70521E9E70621E7E70729D0
:107CE0006ED2DFE801F0DE041B3D54758B000146C7
:107CF0001846FBF7F9FE2860B5F90200B5F9001047
:107D000043F2046201445143090C5043A4F85A1051
:107D1000000CA4F85C00A4F85E8028E1404201B2A7
:107D2000504200B2FBF7E0FE2860B5F9020043F2D2
:107D300004614143090CA4F85A10B5F90010084435
:107D400043F204614843000CA4F85C00A4F85E8090
:107D50003BE13046F8F788FF01231A4607216CE023
:107D600019461046FBF7C0FE2860A4F85A80B5F902
:107D70000200B5F9001043F2046201445143090CBA
:107D80005043A4F85C10000CA4F85E004CE159428A
:107D9000404209B200B2FBF7A7FE2860A4F85A805F
:107DA000B5F9020043F204614143090CA4F85C10E8
:107DB000B5F90010084443F204614843000C5FE148
:107DC0006FE03046F8F750FF01231A46052134E0F2
:107DD0001146FBF789FE2860B5F9020043F2046101
:107DE0004143090CA4F85A10A4F85C80B5F90010BE
:107DF000084443F204614843000C6CE1504201B274
:107E0000584200B2FBF770FE2860B5F90200B5F9E0
:107E1000001043F2046201445143090CA4F85A10C3
:107E20005043A4F85C80000CA4F85E0083E1304667
:107E3000F8F71AFF01231A4606213846F8F714FF0F
:107E400001213046F8F786FE0121384627E050E14F
:107E500080090020342C01409002002014050020ED
:107E60005C0000203401002020040020E0030020FA
:107E7000E7060020140A002080080020A2FEFFFF71
:107E8000D8090020F8080020B4090020002401408F
:107E90000028014002E1D3E0A4E074E047E0F8F7F5
:107EA00059FEB9F80800ABF80000B9F80A00ABF8C1
:107EB0000200B9F81000ABF804004D465E46AB482E
:107EC000F9F70EFDB4F85A00F1880844A4F86000F0
:107ED000B4F85C0031890844A4F86200B4F85E008C
:107EE00071890844A4F86400317EA148012978D042
:107EF00034F85A1F018061884180A18881809C49A3
:107F0000028808310A8042884A80808888809848A0
:107F1000896A0830884795F8320000287ED0F9F742
:107F2000A1F815F8320F401E2870BDE8F09F0146F9
:107F30001846FBF7D9FD2860B5F9020040F68151DB
:107F4000484380136880B5F9001040F681525143D0
:107F500089134218A2F68152524252082980A4F88D
:107F60005E201044A4F85C000844A4F85A000021E4
:107F70003046F8F7EFFD00213846F8F7EBFD012316
:107F80001A460621E5E6404201B2504200B2FBF734
:107F9000ABFD2860B5F9020040F6815148438113DA
:107FA0006980B5F9000040F68152504380130A18E9
:107FB000A2F681525242520828801144A4F85E2051
:107FC000A4F85A100844A4F85C0000213046F8F7E1
:107FD000C1FD00213846F8F7BDFD01231A460521F1
:107FE000B7E6B4E019461046FBF77EFD2860B5F908
:107FF000020040F68151484381136980B5F90000C1
:1080000040F68152504380130A18A2F68152524220
:1080100052082880A4F85A20114400E09AE0A4F8FD
:108020005E100844A4F85C0000213046F8F792FD89
:1080300000213846F8F78EFD01231A460721C0E6D5
:108040005942404209B200B2FBF74EFD2860B5F933
:10805000020040F68151484380136880B5F9001052
:1080600040F68152514389134218A2F6815252427E
:1080700052082980A4F85A201044A4F85C0008444F
:10808000A4F85E0000213046F8F764FD0021384670
:10809000F8F760FD01231A46062192E61146FBF728
:1080A00023FD2860B5F9020040F681514843801352
:1080B0006880B5F9001040F6815251438913421887
:1080C000A2F68152524252082980A4F85C20104442
:1080D000A4F85A000844A4F85E0000213046F8F7DE
:1080E00039FD00213846F8F735FD01231A460521F0
:1080F0009DE6504201B2584200B2FBF7F5FC286001
:10810000B5F9020040F68151484380136880B5F903
:10811000001040F68152514389134218A2F6815251
:10812000524252082980A4F85C201044A4F85E0052
:108130000844A4F85A0000213046F8F70BFD00214E
:108140003846F8F707FD01231A4607216FE634F891
:10815000601FCFE607480088A0F5D04168393FF49A
:10816000E4AEBDE8F05FF9F74FBE000080090020E3
:1081700028000020182C01402DE9F041904C914836
:10818000B4F85A100288511A89B20F296FD30088A7
:10819000A4F85A008C480088DFF83082C0074FF0FE
:1081A00000054FF0010741D0874AD4E90C10243272
:1081B0001388B1EB530F02D21288511A08444FF4BE
:1081C000F371884200D208468149B1FBF0F0616C3E
:1081D000C1F35101084406466064F8F720F9002213
:1081E0007C4BF8F788F84FF040427B4BF8F783F868
:1081F0000E22F8F7EFF8F8F749F9A4F8A40094F87C
:108200006500401CC0B284F86500082834D36C486F
:1082100098F84620001F03789A4201D002704580EA
:108220006E4A13786E4A23B1458021E06564A564E7
:1082300058E0D8F89410A1F5FA618E4211DD616D15
:108240008B1C9E4205DDB0F902100A290DDA491C8B
:1082500006E08E4205DAB0F90210002908DD491E59
:108260004180B0F902000A2802DB177001E0A2E0A9
:108270001570666584F865505A484FF4A542017838
:10828000C1F38101012949D002294AD044F68771FE
:108290002181A4F8A020B0F9243089B24B439B136C
:1082A000A4F89C30B0F90E0000237043B0FBF1F04D
:1082B000A16CC0F3D100C1EBC101C90200EB913048
:1082C000A064F017810341EA9641B003F7F72CFF51
:1082D000B4F8A210C1EBC101C902C00800EB913093
:1082E000A4F8A200616CA06E0844A06694F86C200B
:1082F000521CD2B284F86C20082A05D3C008A4F816
:108300006E0084F86C50A566374A384ED3885806FC
:1083100033D498F80F00022806D02CE043F2045121
:10832000B6E744F24621B3E7B06840F69916B0428A
:1083300021DD94F8380094F88660B0420CD084F8BF
:10834000860094F83D0000F00106C0F3400086422C
:1083500002D1A4F8825004E0B4F88200B0F5966F20
:1083600005D2B4F88200401CA4F8820005E043F076
:108370008000D08001E0A4F88250114894F83F209A
:10838000B0300C2A01D2C57400E0C774174B41F21B
:10839000482641F2504C93F83C400C4B0C2AB3F861
:1083A00082300AD3B14208DB012C06D0614502DDE0
:1083B000002B00D18774BDE8F0818574FBE70000D5
:1083C00034010020F006002000040040900200204C
:1083D0004564BD0100209C40133B3340DE03002078
:1083E000DF030020AC040020000A00201405002058
:1083F0002DE9F041384C394E394F207841F2333174
:10840000C2074FF000050CD0A28962B394F90700AF
:10841000002800DA4042C0B2032829D240F2AE70F0
:108420002AE0A570E5732F4AE571A58192F83830EE
:10843000237220F00800A18040F0020020703D86E9
:108440007560B560F560916C490005D041F68461B6
:10845000A18140F010002070C0B240F001002070F7
:108460006574BDE8F081658120F01000207015E092
:10847000042803D240F6510060810FE0052802D2A3
:1084800040F69910F8E740F6CC42062803D30728B7
:1084900001D3082801D2628100E0618197F89D0034
:1084A00098B9B088102301B2B4F90A003622FCF75B
:1084B000E1F97060F168401AB1680844B060B6F93B
:1084C00000104843C013F0603886388E10B1012088
:1084D000A070C6E7A570C4E7080C00207006002055
:1084E00090020020340100202DE9F041554C2678FF
:1084F000F0077CD05448217A544D90F838008142DE
:108500007BD0534A2346DFF84CC1575C93F90E20C9
:1085100093F90730874203D01CF80170874213D1CA
:1085200046F002065B1C26705BB2E3711CF801107A
:10853000814201D15B1CE37194F90710062901DD2A
:108540000621E171521C1CE0434F17F801C0434F54
:10855000844503D017F801C0844513D126F00206E4
:108560005B1E26705BB2E371795C814201D15B1EB8
:10857000E37194F907306FF005018B4200DAE17185
:10858000521EA273207294F907108A1C042A02D981
:1085900041F68462A2812C4A012912780ADD2B4B14
:1085A00056079B6802D543F0080301E023F0080357
:1085B000AB606070B1F1FF3F09DA5107A96802D5DD
:1085C00021F0080101E041F00801A9606070F9F7AD
:1085D000E5FEA078012810D121488068A3280CDA94
:1085E00094F90700022803DD0220E07105E01EE097
:1085F0006FF00101884200DAE171A089002630B1F4
:10860000401E0004000CA08101D1E671A673E87B36
:1086100004280CD0B5F93010512341220020FCF77A
:1086200029F92886002802D1E07B10B1A670BDE8A8
:10863000F0810C4806700C480670207820F001008C
:108640002070F4E7080C0020340100209002002084
:108650000C910008129100081E9100082491000856
:108660001405002004070020E7060020E73F943DA2
:108670007D3B9A39E1374E36DB34853347321F3143
:108680000B30082F142E2F2D572C8B2BC92A112A73
:108690006229BB28000000368E0300381C07003A10
:1086A0001C07003C8808003E88080040AA0A0042D7
:1086B000AA0A0044AA0A0046CC0C0048CC0C004A86
:1086C000380E004C380E004E380E0050380E005256
:1086D000380E0054380E0056380E0058380E005A26
:1086E000380E005C380E005E380E0060380E0062F6
:1086F000380E0064380E0066380E0068380E006AC6
:108700000000003A8E03003C1C07003E8808004031
:10871000F4090042AA0A0044CC0C0046380E004876
:10872000A40F004A1111004C7D12004E331300506B
:10873000E91300529F140054551500565515005862
:108740005515005A5515005C5515005E551500600D
:1087500055150062551500645515006655150068DD
:108760005515006A5515006C5515006E0000004047
:1087700022020044440400486606004C8808005069
:10878000F4090054600B0058160C005CCC0C00601F
:10879000820D0064380E0068EE0E006C000000349C
:1087A00000000036000000380000003A0000003CE5
:1087B0000000003E000000400000004200000044B5
:1087C00000000046000000480000004A0000004C85
:1087D0000000004E00000050000000520000005455
:1087E00000000056000000580000005A0000005C25
:1087F0000000005E000000600000006200000064F5
:1088000000000066000000684414585858701111A8
:108810005858587041115858487011144858587099
:1088200014115848587099190056991900549919FB
:108830000052991900509919004E9919004C991934
:10884000004A991900489919004699190044991944
:1088500000423D1A0040E11A003E851B003C281CE6
:10886000003ACC1C0038B81E003600200034A3208B
:108870000032EB2100303323002E7A24002C6626B0
:10888000002A512800283D2A0026282C0024B82E32
:108890000022EB3100203333001E1E35001CAE37A2
:1088A000001A00400018004000160040001400406C
:1088B0000012004000100040000E0040000C00407C
:1088C000000A00400008004000060040000400408C
:1088D0000002004000000000010203040500050042
:1088E000010203040104000305020000F00100007E
:1088F00036010000F8000000BA0000007C00000013
:108900007C0000007C00000041141411111444117B
:10891000141441110000290052007B00A400CC0077
:10892000F5001E01470170019901C201EA0113021D
:108930003C0265028E02B602DF02080330035903CF
:108940008203AA03D303FB0324044C0475049D048F
:10895000C504EE0416053E0567058F05B705DF055E
:1089600007062F0657067F06A706CE06F6061E0741
:1089700046076D079507BC07E4070B08320859083E
:108980008108A808CF08F6081D0944096A09910959
:10899000B809DE09050A2B0A520A780A9E0AC40A97
:1089A000EA0A100B360B5C0B820BA80BCD0BF30BFA
:1089B000180C3E0C630C880CAD0CD20CF70C1C0D83
:1089C000410D650D8A0DAF0DD30DF70D1C0E400E38
:1089D000640E880EAC0ECF0EF30E170F3A0F5E0F1B
:1089E000810FA40FC70FEA0F0D1030105310751030
:1089F0009810BA10DD10FF10211143116511871175
:108A0000A911CA11EC110D122E12501271129212EC
:108A1000B312D412F4121513361356137613961399
:108A2000B713D713F613161436145614751494147A
:108A3000B414D314F214111530154E156D158C1590
:108A4000AA15C815E7150516231641165F167C16DC
:108A50009A16B716D516F2160F172C174917661760
:108A60008317A017BC17D917F51711182E184A1815
:108A7000661881189D18B918D418F0180B19261902
:108A800042195D1978199219AD19C819E219FD1921
:108A9000171A311A4C1A661A801A991AB31ACD1A73
:108AA000E61A001B191B331B4C1B651B7E1B971BF7
:108AB000AF1BC81BE11BF91B121C2A1C421C5A1CB1
:108AC000721C8A1CA21CBA1CD21CE91C011D181D98
:108AD000301D471D5E1D751D8C1DA31DBA1DD01DAB
:108AE000E71DFD1D141E2A1E401E571E6D1E831EEF
:108AF000981EAE1EC41EDA1EEF1E051F1A1F2F1F62
:108B0000451F5A1F6F1F841F991FAE1FC21FD71FFB
:108B1000EC1F002000006400C9002D019201F70144
:108B20005B02C00224038903ED035204B6041A0554
:108B30007F05E3054706AB060F077307D7073B081A
:108B40009F0802096609C9092D0A900AF30A560B03
:108B5000B90B1C0C7F0CE20C440DA60D090E6B0E1C
:108B6000CD0E2F0F900FF20F5310B4101511761178
:108B7000D71138129812F8125813B8131814771422
:108B8000D61435159415F3155116B0160E176B172C
:108B9000C91726188318E0183D199919F519511AA3
:108BA000AD1A081B631BBE1B181C731CCD1C261D95
:108BB000801DD91D321E8A1EE31E3B1F921FEA1F15
:108BC00041209820EE2044219A21EF21452299222C
:108BD000EE2242239623E9233C248F24E2243425E9
:108BE0008525D72528267826C82618276827B72759
:108BF00006285428A228EF283D298929D629222A87
:108C00006D2AB82A032B4D2B972BE12B2A2C722C83
:108C1000BB2C022D4A2D912DD72D1D2E632EA82E53
:108C2000EC2E302F742FB82FFA2F3D307F30C0300C
:108C3000013141318131C13100323F327D32BA32AE
:108C4000F73234337033AC33E73322345C34953449
:108C5000CE3407353F357735AE35E4351A365036E4
:108C60008536B936ED36203753378637B737E9378B
:108C7000193849387938A838D738053932395F3941
:108C80008B39B739E2390D3A373A603A893AB23A14
:108C9000DA3A013B283B4E3B733B983BBD3BE03B04
:108CA000043C263C483C6A3C8B3CAB3CCB3CEA3C1D
:108CB000093D273D443D613D7D3D993DB43DCE3D5F
:108CC000E83D013E1A3E323E493E603E763E8C3ED5
:108CD000A13EB53EC93EDC3EEF3E013F123F233F81
:108CE000333F433F513F603F6E3F7B3F873F933F62
:108CF0009E3FA93FB33FBC3FC53FCD3FD53FDC3F83
:108D0000E23FE83FED3FF13FF53FF93FFB3FFD3FDD
:108D1000FF3FFF3FFF3F0000E7382C35002020EFEA
:108D20002037202333202620210000800200040069
:108D30000800100000020004000804000002000403
:108D400000080010002000400080040000000080A7
:108D5000000000400000002000000010000000089B
:108D6000000000040000000200000001000080007C
:108D7000000040000000200000001000000008007B
:108D8000000004000000020000000100008000005C
:108D900000080140000C0140000C0140000C0140A3
:108DA000000C0140000C0140000C0140000C01408F
:108DB000001001400010014000100140001001406F
:108DC000001001400010014000100140001001405F
:108DD0000014014004080140040C0140040C01404F
:108DE000040C0140040C0140040C0140040C01403F
:108DF000040C014004100140041001400410014023
:108E0000041001400410014004100140041001400E
:108E1000041001400414014008080140080C0140FE
:108E2000080C0140080C0140080C0140080C0140EE
:108E3000080C0140080C01400810014008100140D6
:108E400008100140081001400810014008100140BE
:108E50000810014008100140081401400C080140AE
:108E60000C0C01400C0C01400C0C01400C0C01409E
:108E70000C0C01400C0C01400C0C01400C1001408A
:108E80000C1001400C1001400C1001400C1001406E
:108E90000C1001400C1001400C1001400C1401405A
:108EA00010080140100C0140100C0140100C014052
:108EB000100C0140100C0140100C0140100C01403E
:108EC000101001401010014010100140101001401E
:108ED000101001401010014010100140101001400E
:108EE000101401400000000000000000000000001D
:108EF000000000000000000014080140140C0140B4
:108F0000140C0140140C0140140C0140140C0140DD
:108F1000140C0140140C01401410014014100140C5
:108F200014100140141001401410014014100140AD
:108F300014100140141001401414014000000000FE
:108F40000000000000000000000000000000000021
:108F5000FFFFFF0F0FFFFFFFFFF0FFFFFF0FFFFF00
:108F6000FFFFF0FF0FFFFFFFFFF0FFFFFF0FFFFF0F
:108F7000FFF0FFFF0FFFFFFFFFF0FFFFFF0FFFFFFF
:108F8000FFFFF0FFFFFF0FFFFFFFFFF0FFFFFF0FEF
:108F9000FFF0FFFF00000040400000000004000060
:108FA0000040000000000400400000000004000039
:108FB0000040000000040000400000000004000029
:108FC0000040000000000400000040000000000419
:108FD000000000400004000000000080800000004D
:108FE0000008000000800000000008008000000071
:108FF0000008000000800000000800008000000061
:109000000008000000800000000008000000800050
:1090100000000008000000800008000000000020A0
:1090200020000000000200000020000000000200FC
:1090300020000000000200000020000000020000EC
:1090400020000000000200000020000000000200DC
:1090500000002000000000020000002000020000CC
:1090600000000060600000000006000000600000DA
:109070000000060060000000000600000060000024
:109080000006000060000000000600000060000014
:109090000000060000006000000000060000006004
:1090A000000600000080020004000800100000021A
:1090B0000004000804000002000400080010002062
:1090C0000040008004000000FF7FFFFFFDFFFFFF66
:1090D000FBFFFFFFF7FFFFFFEFFFFFFFFFFDFFFFBE
:1090E000FFFBFFFFFFF7FFFFFBFFFFFFFFFDFFFFA2
:1090F000FFFBFFFFFFF7FFFFFFEFFFFFFFDFFFFFBC
:10910000FFBFFFFFFF7FFFFFFBFFFFFF0102030425
:109110000500020304050001030405000102050027
:109120000102030404050001020355050010AA1AF8
:1091300055250030AA3A0000AA0A55150020AA2A8F
:109140005535FF3F6491000800000020180700001B
:10915000E80600085492000818070020B009000033
:109160008063000845020406082D0102030404057B
:10917000400607080913E12B1B08F50421135515B8
:109180002A40061908019313F53D1408193E1B08DF
:109190001504012D17020604050103148020FF8B1E
:1091A000AA0A02019C15AA0A551500085920AA2AE4
:1091B0005535FF3F072903010504060203127C15FC
:1091C00073FFFF04FF8080010125025B6402130A24
:1091D00013ED6612081201100C05040602030101CA
:1091E00003070505280B0102030402060703030415
:1091F0000C3D0706040509191F1919043105060657
:109200004BAA1A024B381E026910312E40FD3969F3
:10921000260211042F405F020C26405B262ACD5502
:10922000155515123902017F0316D0071AFF0101E7
:109230003B0261AA6C080108A80916C49122031216
:10924000100A17401C12600A16901B01491301678F
:049250000200080010
:020000040800F2
:10FC00004A46545A594D46312D4E3330202020203B
:10FC1000050406020301AA0AAA0AAA0AAA0AAA0A4B
:10FC2000AA0ADE3F00100000FF0131000201664613
:10FC300000400040513800400040004000400101B9
:10FC400000400040FF387B257B257B25FF003333B8
:10FC50000201401F00016626B81E6626FFFFFFFF57
:10FC6000FFFF01010100010000000200000202008C
:04FC70000000AA5591
:04000005080000ED02
:00000001FF
